:020000040800F2
:10000000A8070024B1020008E5620008EF560008C6
:10001000E1620008190A0008C97600080000000023
:10002000000000000000000000000000C967000898
:100030009D0C000800000000E9620008CB67000882
:10004000CB020008CB020008CB020008CB0200085C
:10005000CB020008CB020008CB020008CB0200084C
:10006000CB020008CB020008CB020008CB0200083C
:10007000CB020008CB020008CB020008CB0200082C
:10008000CB020008CB020008CB020008CB0200081C
:10009000CB020008CB020008CB020008CB0200080C
:1000A000CB020008CB020008CB020008CB020008FC
:1000B000CB020008CB020008CB020008CB020008EC
:1000C000CB020008CB020008CB020008CB020008DC
:1000D000CB020008CB020008CB020008CB020008CC
:1000E000CB020008CB02000800000000CB02000891
:1000F000CB020008CB020008CB020008CB020008AC
:10010000CB020008CB020008CB020008CB0200089B
:10011000CB020008CB020008CB020008CB0200088B
:10012000CB020008CB020008CB020008CB0200087B
:10013000CB020008CB020008CB020008CB0200086B
:1001400000000000000000000000000000000000AF
:10015000CB020008CB020008CB020008CB0200084B
:10016000CB020008CB020008CB020008CB0200083B
:10017000CB020008CB020008CB020008CB0200082B
:10018000CB020008CB020008CB020008CB0200081B
:10019000CB020008CB020008CB020008CB0200080B
:1001A000CB020008CB020008CB020008CB020008FB
:1001B000CB020008CB020008CB020008CB020008EB
:1001C000CB020008CB020008CB020008CB020008DB
:1001D000CB020008CB020008CB020008CB020008CB
:1001E000CB020008CB020008CB020008CB020008BB
:1001F000CB020008CB020008CB020008CB020008AB
:10020000CB020008CB020008CB020008CB0200089A
:10021000CB020008CB020008CB020008CB0200088A
:10022000CB020008CB020008CB020008000000004F
:10023000CB020008CB02000800000000CB0200083F
:10024000CB020008CB020008CB020008CB0200085A
:10025000CB020008CB020008CB020008CB0200084A
:10026000CB020008CB020008CB020008CB0200083A
:10027000CB020008CB020008CB02000800000000FF
:10028000CB020008CB020008CB02000800000000EF
:1002900000000000CB020008DFF810D000F088FA60
:1002A00000480047999A0008AFF30080A80700248F
:1002B0000648804706480047FEE7FEE7FEE7FEE700
:1002C000FEE7FEE7FEE7FEE7FEE7FEE7A9680008B7
:1002D000990200082DE9F05F0546002092469B46F2
:1002E00088460646814640241BE02846414647464C
:1002F000224600F095F853465A46C01A914110D351
:1003000011461846224600F07CF82D1A67EB0108CA
:100310004F4622460120002100F073F817EB000938
:100320004E41201EA4F10104DFDC484631462A4636
:100330004346BDE8F09F2DE9F0410024061B254609
:1003400071F1000605DA01240027D0EB070067EB06
:100350000101161E73F1000605DA0027D2EB070231
:10036000012567EB0303FFF7B5FF86460E461746E8
:100370009C46AC4204D00025D0EB050E65EB01068F
:1003800024B10020D2EB000760EB030C704631462D
:100390003A466346BDE8F081D2B201E000F8012B95
:1003A000491EFBD270470022F6E710B513460A46F5
:1003B00004461946FFF7F0FF204610BD30B504464D
:1003C0000020034600E05B1C934203D2E05CCD5C5E
:1003D000401BF8D030BD30B50B460146002020222E
:1003E000012409E021FA02F59D4205D303FA02F542
:1003F000491B04FA02F52844151EA2F10102F1DCA2
:1004000030BD202A04DB203A00FA02F100207047B8
:100410009140C2F1200320FA03F319439040704742
:10042000202A04DB203A21FA02F00021704721FA49
:1004300002F3D040C2F120029140084319467047B0
:100440002DE9FE4F804681EA0300C00F0C46009064
:1004500021F0004123F00045B8EB0200A94105D28C
:100460004046214690461C460B46024623F000407B
:10047000104347D0270DC7F30A00C3F30A51029077
:10048000401A019040286BDAC3F3130040F4801B3C
:100490000098924620B10023D2EB030A63EB0B0BCA
:1004A00001985946C0F140025046FFF7AAFF0646A0
:1004B0000D4650465946019A00F08CF910EB0800A1
:1004C0006141002487EA115284EAE7731A4340D05D
:1004D000009A62B3019A012A4FEA075215DC001B09
:1004E00061EB02014FF0004202EA0752CDE90042FF
:1004F000001C41F5801132462B4600F08CF903B008
:10050000BDE8F08F40462146F9E7001B61EB020190
:10051000001C41F5801300185B412018A2F500175C
:1005200047EB030140EAD570B6196D4111E06D0843
:100530004FEA360645EAC0754FEA0752001B61EBE9
:100540000201001C41F5801149084FEA30000019F2
:10055000514132462B4603B0BDE8F04F00F04CB994
:100560000098012240000023D0EB020263EBE0730D
:10057000009821464FEAE074B8EB000061EB0401FB
:10058000E9E783F000435BE781F0004158E72DE99C
:10059000FE4F81EA030404F0004421F0004100947E
:1005A0004FF0000B23F0004350EA01045ED052EA02
:1005B00003045BD0C3F30A54C1F30A552C44A4F2DC
:1005C000F3340194A0FB0254C1F3130141F48011F0
:1005D000C3F3130343F4801301FB024400FB034EF7
:1005E000840A970A44EA815447EA8357A4FB0768C0
:1005F00002958D0A05FB07854FEA932C04FB0C54EA
:100600002705029D4FEA065847EA1637B5EB08055D
:100610006EEB070C870E920E47EA811742EA8312AF
:10062000A7FB0201B6EB0B0164EB00042B0D43EAC0
:100630000C335E1844EB1C50DA465146E7FB0201CE
:10064000C5F313044FEA0B3343EA14534FEA043261
:10065000019C43EA0603A4F10C040294009CCDE93A
:1006600000B400F0D8F803B0BDE8F08F00200146D8
:10067000F9E72DE9F04D81EA030404F0004B21F085
:10068000004514464FF0000A23F0004150EA0502ED
:1006900020D054EA01021DD0C5F30A570246C5F323
:1006A0001303C1F31300C1F30A5640F4801543F459
:1006B0008013A7EB0608101BD64608F2FD3873EB33
:1006C000050002D308F1010801E092185B41B8F17E
:1006D000000F03DA00200146BDE8F08D00204FF442
:1006E0008011064684460EE0171B73EB050705D301
:1006F000121B63EB050306434CEA010C49084FEA61
:10070000300092185B4150EA0107EDD152EA030034
:1007100012D082EA040083EA0501084305D0101BC9
:10072000AB4106D20122002306E000224FF0004335
:1007300002E06FF0010253101AEB06004CEB085177
:1007400010EB0A0041EB0B01BDE8F04D00F054B88E
:10075000C1F30A52C1F3130140F2FF3341F4801197
:100760009A4202DA00200146704740F233439A422F
:10077000A2F2334202DC5242FFF752BEFFF741BE03
:1007800030B5041E71F1000404DB4FF00044404218
:1007900064EB0101141E73F1000405DB1C464FF0ED
:1007A0000043524263EB0403994208BF904230BDBC
:1007B000064C074D06E0E06840F0010394E80700AE
:1007C00098471034AC42F6D3FFF76AFD58BE0008D4
:1007D00078BE0008202A06DBCB17203A41FA02F047
:1007E00043EAE07306E041FA02F3D040C2F120028E
:1007F000914008431946704710B5141E73F1000468
:1008000008DA401C41F1000192185B411A4301D102
:1008100020F0010010BD2DE9F04D92469B4611B12C
:10082000B1FA81F202E0B0FA80F220329046FFF78E
:10083000E8FD04460F4640EA0A0041EA0B01534630
:100840005A46084313D0114653EA010019D0C8F1A3
:1008500040025046FFF7E4FD05460E465046594615
:100860004246FFF7CEFD084305D0012004E02046B4
:100870003946BDE8F08D0020054346EAE0762C437A
:1008800037430A986305E40AA0EB08000022FD0A3A
:1008900044EA47540A3002D500200146E9E7010541
:1008A00010196941DDE9084500196941BDE8F04DBD
:1008B000A2E7000070B504464F492068884203D083
:1008C0004E492068884208D14D48006800F4403005
:1008D00008B1012009E0002007E04A48006800F460
:1008E000403008B1012000E00020B8B103F07CFDE9
:1008F00005466068B0F5803F06D0B0F5003F04D0F3
:10090000B0F5403F08D105E000BF6068000CB5FBC2
:10091000F0F502E0AD0800E000BF2BE04FF400204E
:10092000002102F0C5F805466068C0F31101F9B96D
:1009300080140C281CD2DFE800F01B060708090A07
:100940000B111315171900BF00BF00BF00BF00BF78
:100950006068800C4000B5FBF0F50AE02D0908E066
:100960006D0906E0AD0904E0ED0902E02D0A00E0A2
:1009700000BF00BF00F0C0FF41F20301884210D861
:100980002148854206D92068806840F4807021683B
:1009900088602FE02068806820F48070216888607B
:1009A00028E06D081948854206D82068806820F440
:1009B0004070216888601DE01548854208D820688D
:1009C000806820F4407040F480702168886011E0F5
:1009D0001048854208D82068806820F4407040F4B0
:1009E00000702168886005E02068806840F44070ED
:1009F0002168886070BD0000002002400021024094
:100A00000823024008630258002D3101105E5F0088
:100A100020BCBE0040787D0100BFFEE7F0B585B088
:100A20003D4803901020ADF810000C208DF8120006
:100A300001208DF8130003A809F0EEFA06463146AE
:100A400036A006F043FE002E63D178200AF0F6F8B7
:100A500010B936A006F03AFE782009F0C3F910B9B3
:100A60003BA006F033FE32200AF09AF810B942A0FB
:100A700006F02CFE002002900190009002A809F0E0
:100A8000BBFA01A809F03EFA684609F0E3F99DF8BF
:100A90000030BDF80420BDF8081041A006F016FE95
:100AA00008F006F810B949A006F010FE544C204694
:100AB00008F0CAFF0546E01C08F0C6FF45EAC00082
:100AC00085B2A01D08F0C0FF45EA801085B200BFC6
:100AD0002F46384608F048FA10B94AA006F0F6FD4D
:100AE00040F2731007F08CFE10B950A006F0EEFD36
:100AF000322008F069F910B956A006F0E7FD0AF0B7
:100B000045F9012009F048FF10B95BA006F0DEFDB1
:100B100000BF05B0F0BD00001D9900086D70755F45
:100B2000696E69742C2025640D0A00006D70755F74
:100B30007365745F73656E736F7220636F6D706C35
:100B4000657465202E2E2E2E2E2E0D0A000000001C
:100B50006D70755F636F6E6669677572655F6669F4
:100B6000666F20636F6D706C657465202E2E2E2E5F
:100B70002E2E0D0A000000006D70755F7365745FA6
:100B800073616D706C655F7261746520636F6D7009
:100B90006C657465202E2E2E2E2E2E0D0A00000060
:100BA0006779726F5F726174652025642C206779A4
:100BB000726F5F6673722025642C20616363656CBD
:100BC0005F6673722025640D0A000000646D705F1B
:100BD0006C6F61645F6D6F74696F6E5F647269766C
:100BE00065725F6669726D7761726520636F6D70A3
:100BF0006C657465202E2E2E2E2E2E0D0A00000000
:100C00002D000024646D705F7365745F6F72696599
:100C10006E746174696F6E20636F6D706C6574655E
:100C2000202E2E2E2E2E2E0D0A000000646D705FD9
:100C3000656E61626C655F6665617475726520637F
:100C40006F6D706C657465202E2E2E2E2E2E0D0A63
:100C500000000000646D705F7365745F6669666FA5
:100C60005F7261746520636F6D706C657465202EB2
:100C70002E2E2E2E2E0D0A006D70755F7365745F1B
:100C8000646D705F737461746520636F6D706C6503
:100C90007465202E2E2E2E2E2E0D0A00704772B651
:100CA00000BFFEE72DE9F04399B004460E464FF031
:100CB0000008306800B100BF00BF94F85000012860
:100CC00003D1022019B0BDE8F083012084F8500060
:100CD00000BF00201590169046492068884202D136
:100CE0004548009001E000200090009850B9606DE8
:100CF00040F02000606500BF002084F8500000BF75
:100D00000120DFE7009804F0F0FF0746206804F0B8
:100D1000ECFF002861D1002F5FD13649206888425E
:100D200003D035492068884201D1344800E0344876
:100D30000546306858B3A86820F4404071680843FD
:100D4000A8602C492068884203D02B49206888423B
:100D500001D12A4800E02A482849884209D125487B
:100D600004F0B4FF8146244804F0B0FF49EA0000D3
:100D700002E0244804F0AAFF70BBB1683068084361
:100D8000A96840F61F7291430843A8602BE0A86849
:100D900020F44040A86017492068884203D01649D3
:100DA0002068884201D1154800E01548134988425F
:100DB00009D1104804F08AFF81460F4804F086FFED
:100DC00049EA000002E00F4804F080FF20B9A8685B
:100DD00040F61F718843A86005E0606D40F0200078
:100DE00060654FF0010800BF002084F8500000BF8C
:100DF000404667E7002002400021024000230240F5
:100E000000630258006002582DE9F84F04460D4671
:100E10004FF0000A0020009094F83800012800D11B
:100E200000E000BFFA49E868884200D00EE0F949C6
:100E30002068884200D100BFF7492068884200D16D
:100E400000BFF6492068884200D100BF00BF94F877
:100E50005000012802D10220BDE8F88F012084F85B
:100E6000500000BF206804F03BFF00287ED12868B6
:100E700000F00040A8B92068C1692868C0F31300D9
:100E800018B92868C0F3846004E0286890FAA0F0DC
:100E9000B0FA80F000F01F0201209040014320686A
:100EA000C1612168D5E9002001F1300CC0F3012BAC
:100EB0000CEB8B03D3F800C000F01F0E4FF01F0B9C
:100EC0000BFA0EFB2CEA0B0C00F01F0BC2F3846E26
:100ED0000EFA0BFE4CEA0E0CC3F800C000BF2068EF
:100EE00004F0FEFE8146206804F0E6FE8046B9F17B
:100EF000000F6FD1B8F1000FFBD1AA6829682068F4
:100F000004F0F8FEC648006800F07040B0F1805F61
:100F100007D168692168C968C1F382014900884026
:100F200014E02068C06800F0100038B968692168D2
:100F3000C968C1F382014900884007E068692168F7
:100F4000C96801F0100189084900884007462869EE
:100F5000042840D020682A68296900F1600C0CEB55
:100F60008103D3F800C00CF0004C00E0D0E102F0A7
:100F7000F84B4BEA070B4CEA0B0CC3F800C000BF60
:100F800020686A7E2969012A01D1D20700E0002287
:100F9000134600F1600C0CEB8102D2F800C02CF07B
:100FA000004C4CEA030CC2F800C000BF20682B7E46
:100FB0002969012B01D1DB0200E000231A460369F5
:100FC00023F4F04301F01F0C02FA0CFC43EA0C037B
:100FD000036100BF37E02068006E00F0F840297818
:100FE000B0EB816F05D12068006E20F000402168D1
:100FF00008662068406E00F0F8402978B0EB816FF9
:1010000005D12068406E20F00040216848662068C5
:10101000806E00F0F8402978B0EB816F05D1206830
:10102000806E20F00040216888662068C06E00F065
:10103000F8402978B0EB816F05D12068C06E20F0B0
:1010400000402168C866206804F03BFE002872D189
:101050002068EA682968D0F8C030C1F3130C23EA8D
:101060000C0302F0180BDFF8BCC12CFA0BFC0CEAE5
:10107000010C43EA0C03C0F8C03000BF6449E868C3
:1010800088427DD12B68C3F313031BB92B68C3F3CC
:10109000846304E02B6893FAA3F3B3FA83F35B1C35
:1010A00003F01F03092B3ED82B68C3F313031BB9AE
:1010B0002B68C3F3846304E02B6893FAA3F3B3FAB9
:1010C00083F35B1C03F01F034FF0010C0CFA03FCCD
:1010D0002B68C3F313031BB92B68C3F3846304E0C9
:1010E0002B6893FAA3F3B3FA83F35B1C03F01F039B
:1010F0004CEA836C2B68C3F313031BB92B68C3F34F
:10110000846304E02B6893FAA3F3B3FA83F35B1CC4
:1011100003F01F0303EB43034FF0000B4BEA0353B1
:101120004CEA030341E02B68C3F3130323B92B6894
:10113000C3F3846305E0A9E02B6893FAA3F3B3FA41
:1011400083F35B1C03F01F034FF0010C0CFA03FC4C
:101150002B68C3F313031BB92B68C3F3846304E048
:101160002B6893FAA3F3B3FA83F35B1C03F01F031A
:101170004CEA836C2B68C3F313032BB92B6800E094
:1011800018E0C3F3846304E02B6893FAA3F3B3FA83
:1011900083F35B1C03F01F030A3B03EB43034FF095
:1011A000007B4BEA03534CEA03031946AA68206804
:1011B00004F0A0FD286800F00040002866D0154A21
:1011C0002168914203D0144A2168914201D1164905
:1011D00000E016490846816801F0E07600BF0D493D
:1011E0002068884203D00C492068884201D10E480B
:1011F00000E00E480C4988421AD1064804F061FD0F
:101200008346054804F05DFD4BEA000013E0000052
:101210000000FF4700200240002102400060025809
:101220000010005CFFFF0F00002302400063025823
:101230003E4804F046FDE8BB3D492868884226D177
:1012400006F4000018BB39492068884266D1394B42
:1012500022689A4203D0384B22689A4201D1374A19
:1012600000E0374A104646F4000104F057FD3548C7
:1012700000683549B0FBF1F0401C4000009002E0EE
:101280000098401E009000980028F9D146E02F49B0
:101290002868884219D106F08070B0B923492068C7
:1012A00088423BD1234B22689A4205D0224B2268C8
:1012B0009A4200E025E001D1204A00E0204A104691
:1012C00046F0807104F02AFD28E021492868884210
:1012D00024D106F4800008BB1449206888421DD13F
:1012E000144B22689A4203D0134B22689A4201D1D0
:1012F000124A00E0124A104646F4800104F00EFD46
:101300000CE0606D40F0200060654FF0010A05E0E0
:10131000606D40F0200060654FF0010A00BF0020C2
:1013200084F8500000BF504696E500000060025867
:10133000000084CB00200240002102400023024034
:101340000063025854000024400D0300000052C7FF
:101350000000B8CF2DE9F84F04464FF000090020F7
:10136000009014B90120BDE8F88FE06818B1207F23
:10137000012800D100BF606D30B9204600F030F97F
:101380000020A06584F8500020688168C1F3407196
:1013900031B120688168874A1140816000BF00BF79
:1013A000206804F098FCA8B920688168824A11403E
:1013B00041F08051816000BF804800688049B0FBE7
:1013C000F1F0401C009002E00098401E0090009850
:1013D0000028F9D1206804F07EFC48B9606D40F027
:1013E00010006065A06D40F00100A0654FF001099C
:1013F000206804F075FC0646606D00F010000028BF
:101400007ED1002EFCD1606D20F4807040F002008F
:101410006065206804F055FC78BB6A492068884202
:1014200003D069492068884201D1684800E06848D3
:101430006649884209D1634804F043FC8246624809
:1014400004F03FFC4AEA000002E0624804F039FC84
:1014500098B95C4B22689A4203D05B4B22689A424F
:1014600001D15A4A00E05A4A10466168826822F463
:101470007C120A43826000BF00BF00F03DFA41F2D7
:10148000030188420ED9A06810280BD1607D216B22
:1014900041EA4030A168084340F00C01207F41EA56
:1014A000004508E0607D216B41EA4030A1680843B7
:1014B000217F40EA0145207F012803D1208C401E76
:1014C00045EA4045606A28B1A08C00F47870A16AB2
:1014D000084305432068C0683F4908402843216805
:1014E000C860206804F0FCFB8046206804F0E4FB40
:1014F0000746B8F1000F3BD1D7BB207DE16A00E081
:1015000050E041EA80352068C06844F20301884316
:1015100028432168C86094F83800012817D1606A10
:1015200008B1A06A00B900BFA08F401E012141EAA6
:101530000041206C0843616C0843A16C084321689A
:101540000969264A114008432168086105E02068BE
:10155000006920F00100216808612068006920F01E
:101560007040616B0843216808612046FFF7A2F9CB
:10157000E068012809D12068006B20F00F00A16904
:10158000491E08432168086305E02068006B20F0CD
:101590000F0021680863606D20F0020040F0010038
:1015A000606505E0606D40F0100060654FF0010976
:1015B0004846D8E6C0FFFF5FC0FFFF7F540000240D
:1015C000400D0300002002400021024000230240A1
:1015D000006302580060025803C0F0FF1EF800FCD0
:1015E00010B5B8B00446142132A8FEF7DCFEC021C5
:1015F00002A8FEF7D8FE3049206888425AD14FF43D
:1016000000210020CDE90210042004900921059159
:101610000221069107910891C021099120210A9188
:101620004FF440610B9100202B9002A801F098FE2E
:1016300008B1FFF734FB00BF2048006840F02000ED
:101640001E4908600846006800F02000019000BFB5
:1016500000BF00BF19480830006840F0010017497A
:10166000083108600846006800F00100019000BFE2
:1016700000BF00BF0846006840F00400086008464C
:10168000006800F00400019000BF00BFC02032904D
:10169000032033900020349032A9094800F028F844
:1016A00030203290032033900020349032A9054836
:1016B00000F01EF838B010BD00200240D844025897
:1016C000000002580008025870B5044600F01AF9EC
:1016D00006462546681C10B104480078054400BF42
:1016E00000F010F9801BA842FAD370BD500000240E
:1016F000F8B502460B4600216F4DD7E001278F4019
:101700001E6806EA0704002C72D01E7906F0030654
:10171000012E04D01E7906F00306022E13D1906824
:101720004F000326BE40B0434F00DE68BE4030434A
:101730009060506801268E40B0431E79C6F30016B3
:101740008E40304350601E7906F00306032E09D008
:10175000D0684F000326BE40B0434F009E68BE4095
:101760003043D0601E7906F00306022E13D1CF0855
:1017700002F1200656F827004E07F70E0F26BE404E
:10178000B0434F07FF0E1E69BE403043CF0802F141
:10179000200646F8270010684F000326BE40B043DD
:1017A0001E7906F003064F00BE40304310605E68AD
:1017B00006F44036002E78D000BF404E366846F022
:1017C00002063E4F3E603E46366806F00206009630
:1017D00000BF00BF3A4E8F0856F827008E07370F1C
:1017E0000F26BE40B043374EB24202D100262EE053
:1017F0005BE0354EB24201D1012628E0334EB242C1
:1018000001D1022623E0324EB24201D103261EE06E
:10181000304EB24201D1042619E02F4EB24201D11E
:10182000052614E02D4EB24201D106260FE02C4EC3
:10183000B24201D107260AE02A4EB24201D108265F
:1018400005E0294EB24201D1092600E00A268F07A1
:101850003F0FBE4030431A4E8F0846F827004FF026
:10186000B0463068A0435E6806F4801606B1204397
:101870004FF0B04630607068A0435E6806F4001612
:1018800006B120434FF0B04670606868A0435E68C0
:1018900006F4003606B1204368602868A0435E68FD
:1018A00006F4803606B120432860491C1E68CE40ED
:1018B000002E7FF423AFF8BD80000058F444025896
:1018C000080400580000025800040258000802589A
:1018D000000C025800100258001402580018025858
:1018E000001C025800200258002402580AB18161ED
:1018F00001E00B048361704701480068000C7047E9
:101900000010005C01480068704700004800002497
:10191000024692F8410020282DD100BF92F84000E5
:10192000012801D102207047012082F8400000BF49
:10193000242082F841001068006820F0010013683C
:1019400018601068006820F48050136818601068F0
:1019500000680843136818601068006840F00100D0
:1019600013681860202082F8410000BF002082F830
:10197000400000BFD7E70220D5E710B502460B466E
:1019800092F8410020282AD100BF92F84000012897
:1019900001D1022010BD012082F8400000BF2420A8
:1019A00082F841001068006820F00100146820608F
:1019B0001068016821F4706141EA03211068016038
:1019C0001068006840F0010014682060202082F850
:1019D000410000BF002082F8400000BFDAE702208B
:1019E000D8E7000008B500BF0949096841F00201C5
:1019F000074A11601146096801F00201009100BF19
:101A000000BF044909680143024A116008BD000093
:101A1000F44402580404005810B504460CB90120DF
:101A200010BD94F8410028B9002084F840002046F9
:101A300000F0D8F9242084F841002068006820F0E4
:101A4000010021680860606820F07060216808610A
:101A50002068806820F4004021688860E0680128E0
:101A600005D1A06840F400402168886004E0A068C7
:101A700040F4044021688860E068022806D12068AC
:101A8000406840F400602168486005E020684068D4
:101A900020F40060216848602068406813490843CA
:101AA000216848602068C06820F400402168C86050
:101AB000D4E904010843A16940EA01202168C86013
:101AC000D4E907010843216808602068006840F0F5
:101AD00001002168086000206064202084F8410033
:101AE0000020206384F8420000BF99E700800002D4
:101AF0002DE9F8430446894616461F46DDF8208046
:101B000094F84100202873D100BF94F840000128C8
:101B100002D10220BDE8F883012084F8400000BF14
:101B2000FFF7F0FE054619230122D1032046009558
:101B300003F0A8FE08B10120ECE7222084F8410060
:101B4000102084F84200002060646662678560634C
:101B5000608DFF280CD9FF2020853C48009094F828
:101B600028204FF080734946204603F06FFE0BE0BB
:101B7000608D20853548009094F828204FF0007340
:101B80004946204603F062FE3FE02A464146204691
:101B900003F0BAFE08B10120BCE72068406A616A20
:101BA0000870606A401C6062208D401E2085608D38
:101BB000401E6085608D40B3208D30BB43460022BF
:101BC00080212046009503F05DFE08B10120A1E7C9
:101BD000608DFF280DD9FF2020850020009094F80B
:101BE00028204FF080734946204603F02FFE0CE07A
:101BF0002AE0608D20850020009094F828204FF086
:101C000000734946204603F021FE608D0028BCD1B8
:101C10002A464146204603F0D9FE08B1012079E763
:101C200020202168C861206840680949084021686F
:101C30004860202084F84100002084F8420000BF62
:101C400084F8400000BF65E7022063E700240080BD
:101C500000E800FE2DE9F84F04468A4617469846EC
:101C6000DDF8289094F84100202878D100BF94F83E
:101C70004000012802D10220BDE8F88F012084F83D
:101C8000400000BFFFF73EFE054619230122D103A5
:101C90002046009503F0F6FD08B10120ECE7212075
:101CA00084F84100102084F84200002060646762DC
:101CB000A4F82A806063608DFF2804D9FF20208566
:101CC0004FF0807603E0608D20854FF00076208D08
:101CD000C0B1606A007821688862606A401C6062F6
:101CE000608D401E6085208D401E20853B48009001
:101CF00094F82800401CC2B233465146204603F0F7
:101D0000A5FD08E03548009094F828203346514658
:101D1000204603F09BFD3FE02A464946204603F05B
:101D200085FE08B10120A7E7606A00782168886213
:101D3000606A401C6062608D401E6085208D401E80
:101D40002085608D40B3208D30BB4B460022802122
:101D50002046009503F096FD10B101208CE73AE093
:101D6000608DFF280CD9FF2020850020009094F87A
:101D700028204FF080735146204603F067FD0BE0AA
:101D8000608D20850020009094F828204FF000738B
:101D90005146204603F05AFD608D0028BCD12A46EA
:101DA0004946204603F012FE08B1012064E72020D6
:101DB0002168C86120684068094908402168486076
:101DC000202084F84100002084F8420000BF84F8FD
:101DD000400000BF50E702204EE7000000200080D6
:101DE00000E800FE10B5B8B00446142132A8FEF792
:101DF000DAFAC02102A8FEF7D6FA674920688842BD
:101E000036D108210020CDE90210239002A801F06C
:101E1000A7FA08B1FEF743FF00BF6048006840F032
:101E200002005E4908600846006800F00200019068
:101E300000BF00BF4FF4C0703290122033900020DA
:101E4000349035900420369032A95548FFF750FC65
:101E500000BF52480830006840F400104F49083174
:101E600008600846006800F40010019000BF91E08F
:101E70004C492068884237D108200021CDE9020171
:101E80000020239002A801F06BFA08B1FEF707FFCB
:101E900000BF4248006840F0020040490860084620
:101EA000006800F00200019000BF00BF4FF44060E6
:101EB00032901220339000203490359004203690D8
:101EC00032A93748FFF714FC00BF344808300068D7
:101ED00040F480003149083108600846006800F489
:101EE0008000019000BF55E02F492068884251D101
:101EF00008210020CDE90210239002A801F030FA59
:101F000008B1FEF7CCFE00BF2448006840F0040092
:101F1000224908600846006800F00400019000BFF4
:101F200000BF00BF0846006840F001000860084696
:101F3000006800F00100019000BF00BF4FF4007086
:101F40003290122033900020349035900420369047
:101F500032A91648FFF7CCFB4FF480703290122064
:101F600033900020349035900420369032A91048E8
:101F7000FFF7BEFB00BF09480830006840F40000CE
:101F80000649083108600846006800F40000019026
:101F900000BF00BF38B010BD00540040E0440258FC
:101FA0000004025800580040005C0040000802583D
:101FB00000000258034800680349097808440149B1
:101FC00008607047480000245000002410B503202A
:101FD00000F0A8F802F052FA10490968C1F3032191
:101FE0000F4A515C01F01F0120FA01F40B48006810
:101FF00000F00F001146085C00F01F0024FA00F00A
:1020000008490860084804600F2000F00FF808B184
:10201000012010BD00F036F80020FAE718440258FD
:1020200006BD0008580000245400002470B5044682
:102030001148007808B9012070BD0F4800784FF4AE
:102040007A71B1FBF0F00D490968B1FBF0F5284653
:1020500002F056FF08B10120EEE7102C07D2002253
:102060002146501E00F020F80548046001E00120E0
:10207000E2E70020E0E700005000002454000024C4
:102080004C00002408B500BF0648006840F002007C
:10209000044908600846006800F00200009000BF94
:1020A00000BF08BDF44402582DE9F05F80460D469C
:1020B000164605F033FB074639462A46334601F0FB
:1020C0000700C0F1070ABAF1040F02D94FF0040A61
:1020D00001E0C0F1070AD14600F1040ABAF1070F86
:1020E00002D24FF0000A01E0A0F1030AD4464FF0FB
:1020F000010A0AFA09FAAAF1010A0AEA020A0AFA24
:102100000CFA4FF0010B0BFA0CFBABF1010B0BEAD5
:10211000030B4AEA0B042146404605F007FBBDE8E5
:10212000F09F000000BF00F00702064B19684FF651
:10213000FF031940044B0B4343EA0221014B196092
:1021400000BF70470CED00E00000FA0570B50446D2
:1021500015480068C0F3800048B91348006800F0D3
:102160000700A04201D0012070BD0020FCE70E480E
:10217000006820F0070020430B490860FFF7C2FB0E
:10218000054607E0FFF7BEFB401BB0F57A7F01D99B
:102190000120E9E7044808380068C0F3403000280F
:1021A000F0D00020E0E700000C480258F8B50446E3
:1021B000FFF7A8FB06460CB90120F8BD206A4028AD
:1021C00000D000BF94F8410038B9204600F046F82E
:1021D00041F28831204600F00FF92068006820F4B1
:1021E000F851A068401E41EA002021680860A06CF8
:1021F0003346002220210090204604F076F8054660
:1022000035BB2179E06840EA0160E1690843216A51
:102210000843216809680F4A114008432168086093
:10222000208A616941EA0040A16908432168496840
:10223000094A11400843216848602068006840F05E
:1022400001002168086000206064012084F84100DA
:102250002846B2E72FFFFF00FEF8E0FF10B5B8B048
:102260000446142132A8FEF79EF8C02102A8FEF70A
:102270009AF85A49206888427ED14FF000710020B8
:10228000CDE90210159002A801F06AF808B1FEF736
:1022900006FD00BF5248006840F480405049086085
:1022A0000846006800F48040019000BF00BF00BFF6
:1022B0004B480C30006840F0100049490C31086070
:1022C0000846006800F01000019000BF00BF00BF8A
:1022D0000846006840F0010008600846006800F009
:1022E0000100019000BF00BF00BF0846006840F039
:1022F000020008600846006800F00200019000BF7C
:1023000000BF00BF0846006840F0080008600846AB
:10231000006800F00800019000BF00BF00BF084641
:10232000006840F0040008600846006800F00400FF
:10233000019000BF00BF04203290022033900020A3
:10234000349035900920369032A92648FFF7D0F90D
:10235000022032903390002034903590092036903E
:1023600032A92148FFF7C4F90420329002203390AB
:1023700000203490359000E02EE00920369032A9FC
:102380001A48FFF7B5F94FF40060329002203390FD
:102390000020349035900920369032A91448FFF778
:1023A000A7F94FF4806032900220339000203490DF
:1023B00035900920369032A90E48FFF799F9402050
:1023C0003290022033900020349035900A203690CD
:1023D00032A90648FFF78CF938B010BD0050005202
:1023E000D444025800100258000002580004025859
:1023F000000C0258000802588164704710B501F0C3
:10240000F3FF05490968C1F30211044A515C01F068
:102410001F01C84010BD00002044025806BD00083E
:1024200070B50146844D2D6805F00303824D2D687B
:10243000C5F30510804D2D1D2D6805F001047E4D5E
:102440000C352D68C5F3CC0515FB04F501EE105ACB
:10245000B8EE411AF0EE410A00286FD023B1012BEB
:102460004ED0022B6BD16BE0734D283D2D68C5F328
:1024700040153DB3704D283D2D68C5F3C1066F4D25
:1024800025FA06F201EE102AF8EE411A01EE100AC2
:10249000B8EE411A81EE812A9FED691AC0EE811AC9
:1024A000654D08352D68C5F3080501EE105AB8EEE4
:1024B000411A31EE811AF7EE001A31EE211A22EE9E
:1024C000010A1CE001EE100AB8EE411ADFED5D1AB8
:1024D00081EE812A9FED5A1AC0EE811A564D0835B9
:1024E0002D68C5F3080501EE105AB8EE411A31EE19
:1024F000811AF7EE001A31EE211A22EE010A5BE092
:1025000001EE100AB8EE411ADFED4F1A81EE812A72
:102510009FED4B1AC0EE811A474D08352D68C5F363
:10252000080501EE105AB8EE411A31EE811AF7EEA5
:10253000001A31EE211A22EE010A3DE077E01DE09B
:1025400001EE100AB8EE411A9FED402AC2EE011AC0
:102550009FED3B1A80EE812A374D08352D68C5F373
:10256000080501EE105AB8EE411A32EE011AB7EE24
:10257000002A31EE021A21EE810A1DE001EE100A56
:10258000B8EE411ADFED2F1A81EE812A9FED2C1A49
:10259000C0EE811A284D08352D68C5F3080501EEF7
:1025A000105AB8EE411A31EE811AF7EE001A31EEE8
:1025B000211A22EE010A00BF00BF1F4D08352D6809
:1025C000C5F3462501EE105AB8EE411AF7EE001A8F
:1025D00031EE211AC0EE011ABCEEE11A81ED001AAB
:1025E000154D08352D68C5F3064501EE105AB8EEB5
:1025F000411AF7EE001A31EE211AC0EE011ABCEEB4
:10260000E11A81ED011A0C4D08352D68C5F30665F8
:1026100001EE105AB8EE411AF7EE001A31EE211A07
:10262000C0EE011ABCEEE11A81ED021A03E00025AA
:102630000D604D608D6070BD284402580090D0033D
:10264000000000460024744C0024744A20BCBE4B99
:1026500070B50146844D2D6805F00303824D2D6849
:10266000C5F30530804D2D1D2D68C5F300147E4D3A
:1026700014352D68C5F3CC0515FB04F501EE105A91
:10268000B8EE411AF0EE410A00286FD023B1012BB9
:102690004ED0022B6BD16BE0734D283D2D68C5F3F6
:1026A00040153DB3704D283D2D68C5F3C1066F4DF3
:1026B00025FA06F201EE102AF8EE411A01EE100A90
:1026C000B8EE411A81EE812A9FED691AC0EE811A97
:1026D000654D10352D68C5F3080501EE105AB8EEAA
:1026E000411A31EE811AF7EE001A31EE211A22EE6C
:1026F000010A1CE001EE100AB8EE411ADFED5D1A86
:1027000081EE812A9FED5A1AC0EE811A564D10357E
:102710002D68C5F3080501EE105AB8EE411A31EEE6
:10272000811AF7EE001A31EE211A22EE010A5BE05F
:1027300001EE100AB8EE411ADFED4F1A81EE812A40
:102740009FED4B1AC0EE811A474D10352D68C5F329
:10275000080501EE105AB8EE411A31EE811AF7EE73
:10276000001A31EE211A22EE010A3DE077E01DE069
:1027700001EE100AB8EE411A9FED402AC2EE011A8E
:102780009FED3B1A80EE812A374D10352D68C5F339
:10279000080501EE105AB8EE411A32EE011AB7EEF2
:1027A000002A31EE021A21EE810A1DE001EE100A24
:1027B000B8EE411ADFED301A81EE812A9FED2C1A16
:1027C000C0EE811A284D10352D68C5F3080501EEBD
:1027D000105AB8EE411A31EE811AF7EE001A31EEB6
:1027E000211A22EE010A00BF00BF1F4D10352D68CF
:1027F000C5F3462501EE105AB8EE411AF7EE001A5D
:1028000031EE211AC0EE011ABCEEE11A81ED001A78
:10281000154D10352D68C5F3064501EE105AB8EE7A
:10282000411AF7EE001A31EE211AC0EE011ABCEE81
:10283000E11A81ED011A0C4D10352D68C5F30665BE
:1028400001EE105AB8EE411AF7EE001A31EE211AD5
:10285000C0EE011ABCEEE11A81ED021A03E0002578
:102860000D604D608D6070BD284402580090D0030B
:10287000000000460024744C0024744A20BCBE4B67
:1028800070B50146844D2D6805F00303824D2D6817
:10289000C5F30550804D2D1D2D68C5F300247E4DD8
:1028A0001C352D68C5F3CC0515FB04F501EE105A57
:1028B000B8EE411AF0EE410A00286FD023B1012B87
:1028C0004ED0022B6BD16BE0734D283D2D68C5F3C4
:1028D00040153DB3704D283D2D68C5F3C1066F4DC1
:1028E00025FA06F201EE102AF8EE411A01EE100A5E
:1028F000B8EE411A81EE812A9FED691AC0EE811A65
:10290000654D18352D68C5F3080501EE105AB8EE6F
:10291000411A31EE811AF7EE001A31EE211A22EE39
:10292000010A1CE001EE100AB8EE411ADFED5D1A53
:1029300081EE812A9FED5A1AC0EE811A564D183544
:102940002D68C5F3080501EE105AB8EE411A31EEB4
:10295000811AF7EE001A31EE211A22EE010A5BE02D
:1029600001EE100AB8EE411ADFED4F1A81EE812A0E
:102970009FED4B1AC0EE811A474D18352D68C5F3EF
:10298000080501EE105AB8EE411A31EE811AF7EE41
:10299000001A31EE211A22EE010A3DE077E01DE037
:1029A00001EE100AB8EE411A9FED402AC2EE011A5C
:1029B0009FED3B1A80EE812A374D18352D68C5F3FF
:1029C000080501EE105AB8EE411A32EE011AB7EEC0
:1029D000002A31EE021A21EE810A1DE001EE100AF2
:1029E000B8EE411ADFED301A81EE812A9FED2C1AE4
:1029F000C0EE811A284D18352D68C5F3080501EE83
:102A0000105AB8EE411A31EE811AF7EE001A31EE83
:102A1000211A22EE010A00BF00BF1F4D18352D6894
:102A2000C5F3462501EE105AB8EE411AF7EE001A2A
:102A300031EE211AC0EE011ABCEEE11A81ED001A46
:102A4000154D18352D68C5F3064501EE105AB8EE40
:102A5000411AF7EE001A31EE211AC0EE011ABCEE4F
:102A6000E11A81ED011A0C4D18352D68C5F3066584
:102A700001EE105AB8EE411AF7EE001A31EE211AA3
:102A8000C0EE011ABCEEE11A81ED021A03E0002546
:102A90000D604D608D6070BD284402580090D003D9
:102AA000000000460024744C0024744A20BCBE4B35
:102AB0002DE9F04389B006460F464FF4807186EA4F
:102AC0000100384370D1F748006800F00709B9F1F8
:102AD000050F65D2DFE809F0031221623000F148EA
:102AE0005038006800F00070B0F1007F04D106A8F3
:102AF000FFF796FC079C00E0002453E0E9485038BB
:102B0000006800F00060B0F1006F04D103A8FFF787
:102B10009FFD039C00E0002444E0E2485038006838
:102B200000F00050B0F1005F04D16846FFF7A8FE46
:102B3000009C00E0002435E0DA48001F006800F047
:102B40004055D8485038006800F00400042809D1E6
:102B500045B9D44850380068C0F3C101D24820FAC2
:102B600001F41AE0CF485038006800F48070B0F5E6
:102B7000807F04D1B5F1805F01D1CC4C0DE0C94814
:102B80005038006800F40030B0F5003F04D1B5F1D2
:102B9000005F01D1C64C00E0002403E0C54C01E019
:102BA000002400BFD4E3FFE74FF4007186EA010080
:102BB00038437AD1BB48006800F4E079B9F1800F5E
:102BC0002CD006DCB9F1000F0AD0B9F1400F69D161
:102BD00015E0B9F1C00F63D0B9F5807F62D12CE068
:102BE000B0485038006800F00070B0F1007F04D1A8
:102BF00006A8FFF715FC079C00E0002454E0A94854
:102C00005038006800F00060B0F1006F04D103A8F4
:102C1000FFF71EFD039C00E0002445E0A14850386A
:102C2000006800F00050B0F1005F04D16846FFF783
:102C300027FE009C00E0002436E09A48001F006850
:102C400000F0405597485038006800F00400042810
:102C500009D145B9934850380068C0F3C101924882
:102C600020FA01F41BE08F485038006800F48070AF
:102C7000B0F5807F04D1B5F1805F01D18B4C0EE0BF
:102C800088485038006800F40030B0F5003F05D1A6
:102C9000B5F1005F02D1864C01E006E0002403E0BC
:102CA000844C01E0002400BF52E34FF4806186EAC7
:102CB000010038437BD17B480830006800F460098C
:102CC000B9F5800F2CD006DCB9F1000F0AD0B9F5A8
:102CD000001F69D115E0B9F5C00F63D0B9F5000F39
:102CE00062D12CE06F485038006800F00070B0F1FD
:102CF000007F04D106A8FFF793FB079C00E00024A7
:102D000054E068485038006800F00060B0F1006F8F
:102D100004D103A8FFF79CFC039C00E0002445E0DD
:102D200060485038006800F00050B0F1005F04D1F6
:102D30006846FFF7A5FD009C00E0002436E05948F6
:102D4000001F006800F0405556485038006800F0F9
:102D50000400042809D145B9524850380068C0F32E
:102D6000C101514820FA01F41BE04E485038006878
:102D700000F48070B0F5807F04D1B5F1805F01D19F
:102D80004A4C0EE047485038006800F40030B0F577
:102D9000003F05D1B5F1005F02D1454C01E006E0EE
:102DA000002403E0434C01E0002400BFD0E24FF4D4
:102DB000006186EA0100384373D13A480830006860
:102DC00000F0E069B9F1007F2CD006DCB9F1000F0A
:102DD0000AD0B9F1807F75D115E0B9F1407F6FD08D
:102DE000B9F1806F6ED12CE02E485038006800F0A9
:102DF0000070B0F1007F04D106A8FFF711FB079C1B
:102E000000E0002460E027485038006800F00060CF
:102E1000B0F1006F04D103A8FFF71AFC039C00E097
:102E2000002451E01F485038006800F00050B0F115
:102E3000005F04D16846FFF723FD009C00E00024FA
:102E400042E01848001F006800F04055154850380F
:102E5000006800F00400042809D145B91148503831
:102E60000068C0F3C101104820FA01F427E00D48C2
:102E70005038006800F48070B0F5807F04D1B5F15F
:102E8000805F01D1094C1AE006485038006800F410
:102E90000030B0F5003F11D1B5F1005F0ED1044C08
:102EA0000DE012E0504402580090D00300093D00AC
:102EB00040787D010080BB0004E001E0002403E0D5
:102EC000F74C01E0002400BF42E24FF4805186EA53
:102ED000010038437AD1F348006800F4E048B8F5BF
:102EE000005F2CD006DCB8F1000F0AD0B8F5805F87
:102EF00069D115E0B8F5405F63D0B8F5804F62D175
:102F00002CE0E8485038006800F00070B0F1007F15
:102F100004D106A8FFF784FA079C00E0002454E0DF
:102F2000E0485038006800F00060B0F1006F04D154
:102F300003A8FFF78DFB039C00E0002445E0D9487F
:102F40005038006800F00050B0F1005F04D16846CE
:102F5000FFF796FC009C00E0002436E0D148001FFB
:102F6000006800F04055CF485038006800F0040079
:102F7000042809D145B9CB4850380068C0F3C101D5
:102F8000C94820FA01F41BE0C6485038006800F434
:102F90008070B0F5807F04D1B5F1805F01D1C34C62
:102FA0000EE0C0485038006800F40030B0F5003F33
:102FB00005D1B5F1005F02D1BD4C01E006E000246F
:102FC00003E0B74C01E0002400BFC1E14FF4005121
:102FD00086EA0100384367D1B248006800F4E0286F
:102FE000B8F5403F33D009DCB8F1000F0DD0B8F58B
:102FF000803F0ED0B8F5003F53D119E0B8F5802FCF
:1030000037D0B8F5A02F4CD13FE001F013FA0446B9
:1030100049E0A4485038006800F00060B0F1006F4B
:1030200004D103A8FFF714FB049C00E000243AE05D
:103030009C485038006800F00050B0F1005F04D1A7
:103040006846FFF71DFC019C00E000242BE095483A
:103050005038006800F00400042808D19148503826
:103060000068C0F3C101904820FA01F400E0002498
:1030700019E08C485038006800F48070B0F5807F0B
:1030800001D18A4C00E000240DE0864850380068E9
:1030900000F40030B0F5003F01D1854C00E0002481
:1030A00001E0002400BF53E14FF4002186EA010053
:1030B000384361D17B480830006800F44038B8F1EB
:1030C000000F06D0B8F5803F12D0B8F5003F50D1C0
:1030D0001DE074485038006800F00060B0F1006FE7
:1030E00004D103A8FFF7B4FA039C00E0002442E0F7
:1030F0006C485038006800F00050B0F1005F04D117
:103100006846FFF7BDFB029C00E0002433E0654801
:10311000001F006800F0405562485038006800F019
:103120000400042809D145B95E4850380068C0F34E
:10313000C1015D4820FA01F41AE05A48503800688D
:1031400000F48070B0F5807F04D1B5F1805F01D1CB
:10315000564C0DE053485038006800F40030B0F58C
:10316000003F04D1B5F1005F01D1514C00E00024D3
:1031700001E0002400BFEBE04FF4803186EA01005B
:1031800038432CD14748001F006800F48038B8F15C
:10319000000F03D0B8F5803F1ED10EE041485038F3
:1031A000006800F00070B0F1007F04D106A8FFF7BE
:1031B00037F9079C00E0002410E03A4850380068D6
:1031C00000F00060B0F1006F04D103A8FFF740FAEF
:1031D000059C00E0002401E0002400BFB8E04FF4AB
:1031E000804186EA0100384372D12E4808300068D9
:1031F00000F0E048B8F1405F33D009DCB8F1000FCF
:103200000DD0B8F1805F0ED0B8F1005F5DD119E04C
:10321000B8F1804F37D0B8F1A04F56D14AE0FFF750
:10322000EDF8044653E01F485038006800F0006095
:10323000B0F1006F04D103A8FFF70AFA049C00E084
:10324000002444E017485038006800F00050B0F106
:10325000005F04D16846FFF713FB019C00E00024E7
:1032600035E010485038006800F00400042808D108
:103270000C4850380068C0F3C1010B4820FA01F433
:1032800000E0002423E007485038006800F4807014
:10329000B0F5807F01D1054C00E0002417E017E075
:1032A0000080BB00504402580090D00300093D004C
:1032B00040787D012848006800F40030B0F5003FF8
:1032C00001D1264C00E0002401E0002400BF3FE0D3
:1032D0004FF4004186EA0100384338D11E4850308F
:1032E000006800F04058B8F1000F06D0B8F1805FD8
:1032F0000ED0B8F1005F27D118E01748006800F43D
:103300000030B0F5003F01D1144C00E000241DE076
:103310001148006800F00070B0F1007F04D106A8E9
:10332000FFF77EF8079C00E000240FE00A480068E1
:1033300000F00060B0F1006F04D103A8FFF788F936
:10334000049C00E0002401E0002400BF00E0002411
:10335000204609B0BDE8F0830044025840787D0162
:103360002DE9F04104460025A8464FF00062D4E95B
:10337000001011400020134659404040014331D114
:10338000A06E48B1B0F5801F0DD0B0F5001F11D070
:10339000B0F5401F16D114E0F948006840F4003041
:1033A000F749086010E0022104F1080002F0C4FFB0
:1033B000054609E0022104F1280003F06FF80546F4
:1033C00002E001E0012500BF00BF55B9EC48243000
:1033D000006820F44010A16E0843E94924310860D8
:1033E00000E0A8464FF48073D4E900101940002093
:1033F0005940404001432ED1A06D05281BD2DFE883
:1034000000F0030A11181900DD48006840F400308C
:10341000DB49086011E0002104F1080002F08CFF94
:1034200005460AE0002104F1280003F037F80546BC
:1034300003E002E001E0012500BF00BF55B9D0481C
:103440002430006820F00700A16D0843CC492431E6
:10345000086000E0A8464FF40073D4E9001019405A
:10346000002059404040014334D1E06D802818D0FD
:1034700003DC40B140281DD10CE0C02818D0B0F5C5
:10348000807F17D115E0BE48006840F40030BC4989
:10349000086011E0002104F1080002F04DFF05462C
:1034A0000AE0002104F1280002F0F8FF054603E0DD
:1034B00002E001E0012500BF00BF55B9B04824304B
:1034C000006820F4E070E16D0843AD4924310860E4
:1034D00000E0A8464FF48063D4E9001019400020B2
:1034E00059404040014339D1D4F8A800B0F5800FCD
:1034F0001AD004DC50B1B0F5001F1ED10DE0B0F5BC
:10350000C00F18D0B0F5000F17D115E09C48006827
:1035100040F400309A49086011E0002104F10800ED
:1035200002F00AFF05460AE0002104F1280002F03B
:10353000B5FF054603E002E001E0012500BF00BF42
:103540005DB98F482C30006820F46000D4F8A810D2
:1035500008438B492C31086000E0A8464FF4006214
:10356000D4E9001011400020134659404040014367
:1035700039D1D4F8AC00B0F1007F1AD004DC50B1DE
:10358000B0F1807F1ED10DE0B0F1407F18D0B0F1D6
:10359000806F17D115E07A48006840F40030784910
:1035A000086011E0002104F1080002F0C5FE0546A4
:1035B0000AE0002104F1280002F070FF054603E054
:1035C00002E001E0012500BF00BF5DB96C482C306E
:1035D000006820F0E060D4F8AC10084368492C3152
:1035E000086000E0A8464FF00073D4E900011840DD
:1035F000002158404940084328D1E06CA8B1102868
:1036000004D0202809D0302810D10DE05C48006893
:1036100040F400305A4908600AE0022104F1080031
:1036200002F08AFE054603E002E001E0012500BF4A
:1036300000BF55B952482030006820F03000E16CDE
:1036400008434F492031086000E0A8464FF48053FA
:10365000D4E900101940002059404040014337D1BF
:10366000206EB0F5005F1AD004DC50B1B0F5805F79
:103670001ED10DE0B0F5405F18D0B0F5804F17D1E6
:1036800015E03F48006840F400303D49086011E013
:10369000002104F1080002F04FFE05460AE0002177
:1036A00004F1280002F0FAFE054603E002E001E022
:1036B000012500BF00BF55B931482430006820F40F
:1036C000E040216E08432E492431086000E0A846FE
:1036D0004FF40053D4E900101940002059404040F5
:1036E000014335D1606EB0F5403F1ED007DC68B1B4
:1036F000B0F5803F0BD0B0F5003F19D10EE0B0F52A
:10370000802F13D0B0F5A02F12D110E012E00121CC
:1037100004F1080002F010FE05460BE0012104F15F
:10372000280002F0BBFE054604E003E002E001E0F1
:10373000012500BF00BF55B911482430006820F4AE
:10374000E020616E08430E492431086000E0A8467D
:103750004FF48043D4E9000118400021584049400B
:10376000084337D1D4F8B000B0F1405F20D009DC75
:1037700078B1B0F1805F0DD0B0F1005F1BD110E0E7
:103780002C440258B0F1804F13D0B0F1A04F12D1A9
:1037900010E012E0012104F1080002F0CDFD054621
:1037A0000BE0012104F1280002F078FE054604E058
:1037B00003E002E001E0012500BF00BF4DB9FE4873
:1037C000006820F0E040D4F8B0100843FA490860DF
:1037D00000E0A8464FF40042D4E900101140002058
:1037E000134659404040014329D1206FB0B1B0F198
:1037F000805F03D0B0F1005F11D108E0EE482C38B3
:10380000006840F40030EC492C39086009E00121DF
:1038100004F1080002F090FD054602E001E00125F8
:1038200000BF00BF55B9E4480838006820F0405098
:10383000216F0843E0490839086000E0A8464FF0CE
:103840008072D4E9001011400020134659404040D6
:1038500001432AD1A06CB8B1012804D002280BD0B2
:10386000032812D10FE0D4482C38006840F400300F
:10387000D1492C3908600AE0022104F1080002F065
:103880005BFD054603E002E001E0012500BF00BF4B
:1038900055B9C9480C38006820F00300A16C0843F2
:1038A000C5490C39086000E0A8464FF48002D4E90D
:1038B00000011040002113465840494008437DD183
:1038C000BE48006840F48070BC490860FEF71AF8F2
:1038D000064606E0FEF716F8801B642801D903258A
:1038E00005E0B648006800F480700028F2D000BF00
:1038F00085BBB1481830006800F44070B4F8B410CB
:1039000001F44071884213D0AB481830006820F4AD
:103910004077A9481830006840F48030A649183133
:1039200008600846006820F4803008600846076098
:10393000D4F8B400B0F5807F15D1FDF7E3FF06465B
:1039400009E0FDF7DFFF801B41F28831884202D990
:10395000032507E038E0984818300068C0F34000BD
:103960000028EED000BF55BB00BFB4F8B40000F48F
:103970004070B0F5407F0ED18F484838006820F481
:103980007C518F4AD4F8B400104041EA10108A49A3
:103990004839086007E088484838006820F47C50BF
:1039A000854948390860844818300068B4F8B41074
:1039B000C1F30B0108438049183101E005E001E043
:1039C000086002E0A84600E0A8460122D4E9000110
:1039D00010400021134658404940084330D1E06F61
:1039E00018281AD005DC48B1082808D0102817D1AB
:1039F0000CE0202812D0282812D110E012E001217A
:103A000004F1080002F098FC05460BE0012104F1E6
:103A1000280002F043FD054604E003E002E001E077
:103A2000012500BF00BF55B96348001F006820F0A2
:103A30003800E16F08436049091F086000E0A846AC
:103A40000222D4E9000110400021134658404940A9
:103A5000084329D1A06F062816D2DFE800F003043E
:103A60000B12131412E0012104F1080002F064FCAF
:103A700005460BE0012104F1280002F00FFD054688
:103A800004E003E002E001E0012500BF00BF55B9FA
:103A90004948001F006820F00700A16F084346490D
:103AA000091F086000E0A8460423D4E9001019406B
:103AB000002059404040014329D1D4F89400062801
:103AC00016D2DFE800F003040B12131412E00121F8
:103AD00004F1080002F030FC05460BE0012104F17E
:103AE000280002F0DBFC054604E003E002E001E010
:103AF000012500BF00BF4DB92F48006820F0070026
:103B0000D4F8941008432C49086000E0A84620230C
:103B1000D4E900011840002158404940084337D1FA
:103B2000D4F89000B0F1405F1ED007DC68B1B0F16E
:103B3000805F0BD0B0F1005F19D10EE0B0F1804F83
:103B400013D0B0F1A04F12D110E012E0002104F127
:103B5000080002F0F1FB05460BE0022104F1280009
:103B600002F09CFC054604E003E002E001E00125D0
:103B700000BF00BF5DB91048001F006820F0E040A2
:103B8000D4F8901008430C49091F086000E0A846CB
:103B90004023D4E90010194000205940404001431F
:103BA0003CD1D4F89C00B0F5406F25D00EDCA0B11C
:103BB000B0F5806F12D005E0584402580048025812
:103BC000FFFCFF0FB0F5006F19D10EE0B0F5805F7C
:103BD00013D0B0F5A05F12D110E012E0002104F183
:103BE000080002F0A9FB05460BE0022104F12800C1
:103BF00002F054FC054604E003E002E001E0012588
:103C000000BF00BF4DB9FE48006820F4E050D4F872
:103C10009C100843FA49086000E0A8468023D4E9D4
:103C200000101940002059404040014335D1D4F8DC
:103C3000A000B0F5C04F1ED007DC68B1B0F5005F42
:103C40000BD0B0F5804F19D10EE0B0F5004F13D076
:103C5000B0F5204F12D110E012E0002104F108006D
:103C600002F06AFB05460BE0022104F1280002F095
:103C700015FC054604E003E002E001E0012500BF79
:103C800000BF4DB9DE48006820F46040D4F8A010B1
:103C90000843DB49086000E0A8460823D4E9001087
:103CA0001940002059404040014317D1D4F8840006
:103CB000B0F5805F07D1022104F1280002F0EEFB8D
:103CC00008B14FF00108CE48001F006820F44050B2
:103CD000D4F884100843CA49091F08601023D4E9A6
:103CE00000101940002059404040014315D1D4F83C
:103CF0009800B0F5807F07D1022104F1280002F07E
:103D0000CDFB08B14FF00108BD48006820F44070B9
:103D1000D4F898100843BA4908604FF40022D4E957
:103D2000000110400021134658404940084327D164
:103D3000D4F8A40030B1B0F5803F0AD0B0F5003F10
:103D40000FD10DE0002104F1080002F0F5FA05465C
:103D500009E0022104F1280002F0A0FB054602E080
:103D600001E0012500BF00BF4DB9A548006820F45F
:103D70004030D4F8A4100843A149086000E0A846E8
:103D80004FF48023D4E900011840002158404940F5
:103D900008432DD1D4F88800B0F5801F06D0B0F5C7
:103DA000001F0CD0B0F5401F11D10FE094482C3803
:103DB000006840F4003092492C39086009E0012184
:103DC00004F1280002F06AFB054602E001E001254B
:103DD00000BF00BF5DB98A48001F006820F4401092
:103DE000D4F8881008438649091F086000E0A846F7
:103DF0004FF48032D4E900011040002113465840AE
:103E00004940084325D1206D18B1B0F5803F10D14D
:103E100008E07B482C38006840F4003078492C39A1
:103E2000086008E0022104F1080002F085FA054666
:103E300001E0012500BF00BF55B971480C3800688A
:103E400020F48030216D08436D490C39086000E092
:103E5000A8464FF00052D4E900101140002013464C
:103E600059404040014307D1022104F1280002F0EB
:103E700015FB08B14FF001084FF40033D4E90001FD
:103E80001840002158404940084329D1D4F8800007
:103E9000A0B1B0F5807F06D0B0F5007F0CD0B0F5B2
:103EA000407F0CD109E056482C38006840F40030BF
:103EB00053492C39086004E003E002E001E00125E9
:103EC00000BF00BF5DB94E48001F006820F440707D
:103ED000D4F8801008434A49091F086000E0A8464A
:103EE0004FF48012D4E900101140002013465940CD
:103EF0004040014309D142480838006820F00040A2
:103F0000616F08433E49083908604FF08052D4E998
:103F100000101140002013465940404001430AD18F
:103F200037484838006820F48040D4F8B810084377
:103F30003349483908604FF40012D4E900101140A9
:103F40000020134659404040014309D12C4808380D
:103F5000006820F08070E16E084329490839086044
:103F60004FF08042D4E90010114000201346594020
:103F70004040014311D100BF21484838006820F477
:103F800000401F494839086008460068D4F8BC1052
:103F900008431B494839086000BF4FF00042D4E98C
:103FA000001011400020134659404040014309D100
:103FB00013480C38006820F04050616D08431049E8
:103FC0000C3908604FF40002D4E9001011400020C1
:103FD00013465940404001430AD10948001F006878
:103FE00020F44000D4F88C1008430549091F0860EC
:103FF000012300216068184001224940504001E03F
:1040000058440258014306D104F1080002F094F923
:10401000054605B1A84602220021606810404940CB
:104020005040014307D1012104F1080002F084F956
:10403000054605B1A8460423002061681940042202
:1040400040405140084307D1022104F1080002F02A
:1040500073F9054605B1A846082300216068184099
:10406000082249405040014306D104F1280002F0E3
:1040700015FA054605B1A8461022002160681040D7
:1040800049405040014307D1012104F1280002F0CA
:1040900005FA054605B1A8462022002061681140B6
:1040A00040405140084307D1022104F1280002F0AA
:1040B000F5F9054605B1A846B8F1000F02D1002078
:1040C000BDE8F0810120FBE72DE9F04104460D46F3
:1040D00014B90120BDE8F081BD48006800F00F0070
:1040E000A8420ED2BA48006820F00F002843B84911
:1040F00008600846006800F00F00A84201D00120C7
:10410000E8E7207800F0040004280ED1B1492069C6
:10411000096801F07001884207D9AE48006820F0B4
:10412000700021690843AB490860207800F008005E
:10413000082811D1A749091D6069096801F07001BB
:10414000884209D9A348001D006820F07000616909
:104150000843A049091D0860207800F010001028CD
:1041600011D19C49091DA069096801F4E0618842E8
:1041700009D99848001D006820F4E060A16908434F
:104180009449091D0860207800F02000202811D1F2
:1041900090490831E069096801F07001884209D945
:1041A0008C480830006820F07000E16908438949B4
:1041B00008310860207800F0020002280ED18549FD
:1041C000E068096801F00F01884207D9814800685A
:1041D00020F00F00E16808437E490860207800F075
:1041E0000100002850D07B48006820F47060A1686E
:1041F0000843784908606068022807D17548183874
:104200000068C0F34040F8B9012063E76068032804
:1042100007D1704818380068C0F34060A0B9012089
:1042200058E76068012807D16A4818380068C0F369
:10423000002048B901204DE7664818380068C0F3EF
:10424000800008B9012045E762480838006820F07E
:104250000700616808435F4908390860FDF752FBB1
:10426000064608E0FDF74EFB801B41F2883188428C
:1042700001D903202EE757480838006800F03800BD
:104280006168B0EBC10FEDD1207800F00200022888
:104290000ED15049E068096801F00F01884207D249
:1042A0004C48006820F00F00E16808434949086065
:1042B0004748006800F00F00A8420ED94448006843
:1042C00020F00F002843424908600846006800F0CB
:1042D0000F00A84201D00120FCE6207800F0040085
:1042E00004280ED13B492069096801F07001884219
:1042F00007D23848006820F070002169084335492A
:104300000860207800F00800082811D13149091D03
:104310006069096801F07001884209D22D48001DCA
:10432000006820F07000616908432A49091D08608F
:10433000207800F01000102811D12649091DA0692D
:10434000096801F4E061884209D22248001D006832
:1043500020F4E060A16908431E49091D0860207827
:1043600000F02000202811D11A490831E0690968BD
:1043700001F07001884209D216480830006820F028
:104380007000E169084313490831086000F076F8CD
:1043900010490968C1F303210F4A515C01F01F0164
:1043A00020FA01F70B48006800F00F001146085C86
:1043B00000F01F0027FA00F008490860084807606D
:1043C00008480068FDF732FE8046404682E600005D
:1043D000002000521844025806BD0008580000246E
:1043E000540000244C00002410B500F047F80D499B
:1043F0000968C1F303210C4A515C01F01F0120FA46
:1044000001F40848006800F00F001146085C00F055
:104410001F0024FA00F005490860054804600846BA
:10442000006810BD1844025806BD0008580000245A
:104430005400002400B5FFF7D7FF05490968C1F310
:104440000211044A515C01F01F01C84000BD000088
:104450001C44025806BD000800B5FFF7C5FF05491A
:104460000968C1F30221044A515C01F01F01C840F0
:1044700000BD00001C44025806BD0008F0B5824E85
:10448000366806F0380636B1082E15D0102E15D035
:10449000182E7DD114E07C4E103E3668C6F34016CF
:1044A00046B1794E103E3668C6F3C107774E26FAFC
:1044B00007F000E07548E5E07548E3E07548E1E0A5
:1044C000714E1836366806F003046F4E183636689B
:1044D000C6F305116C4E1C36366806F001056A4EAF
:1044E00024363668C6F3CC0616FB05F601EE106AD4
:1044F000B8EE410A002971D024B1012C50D0022C11
:104500006DD16DE0604E103E3668C6F340163EB386
:104510005D4E103E3668C6F3C1075C4E26FA07F3BF
:1045200001EE103AF8EE411A01EE101AB8EE411AF7
:1045300081EE812A9FED581AC0EE011A524E2036A4
:104540003668C6F3080601EE106AB8EE411A31EE7D
:10455000811AF7EE001A31EE211A62EE010A1EE00E
:1045600001EE101AB8EE411ADFED4C1A81EE812AE5
:104570009FED491AC0EE011A434E20363668C6F345
:10458000080601EE106AB8EE411A31EE811A00E019
:1045900076E0F7EE001A31EE211A62EE010A5BE0D6
:1045A00001EE101AB8EE411A9FED3D2AC2EE011A33
:1045B0009FED391A80EE012A334E20363668C6F355
:1045C000080601EE106AB8EE411A32EE011AB7EE93
:1045D000002A31EE021A61EE810A3DE04EE01DE054
:1045E00001EE101AB8EE411ADFED2E1A81EE812A83
:1045F0009FED291AC0EE011A234E20363668C6F305
:10460000080601EE106AB8EE411A31EE811AF7EE93
:10461000001A31EE211A62EE010A1DE001EE101AB5
:10462000B8EE411A9FED1E2AC2EE011A9FED1A1A2A
:1046300080EE012A144E20363668C6F3080601EED5
:10464000106AB8EE411A32EE011AB7EE002A31EEC6
:10465000021A61EE810A00BF00BF0B4E2036366899
:10466000C6F34626721C01EE102AB8EE411AC0EEBF
:10467000811ABCEEE11A11EE100A00E0002001E000
:10468000034800BF00BFF0BD104402580090D003A3
:1046900000093D0040787D01000000460024744C74
:1046A0000024744A20BCBE4B2DE9F047044614B9DF
:1046B0000120BDE8F087207800F00100002870D0CC
:1046C000FA48006800F03808F8481830D0F8009030
:1046D000B8F1100F06D0B8F1180F0FD109F0030090
:1046E00002280BD1F14810380068C0F34040002880
:1046F0006AD06068002867D10120DAE700BF6068EF
:10470000B0F5803F08D1E9481038006840F48030A7
:10471000E649103908602EE0606868B9E34810384F
:10472000006820F48030E1491039086008460068CC
:1047300020F4802008601EE06068B0F5A02F0DD145
:10474000DA481038006840F48020D84910390860F1
:104750000846006840F4803008600CE0D348103808
:10476000006820F48030D14910390860084600689C
:1047700020F48020086000BF606898B1FDF7C2F89F
:10478000054606E0FDF7BEF8401B642801D903206A
:104790008FE7C64810380068C0F340400028F1D0C9
:1047A00012E012E0FDF7AEF8054606E0FDF7AAF8C4
:1047B000401B642801D903207BE7BC4810380068FF
:1047C000C0F340400028F1D100BF207800F0020083
:1047D000022874D1B548006800F03808B348183092
:1047E000D0F80090B8F1000F05D0B8F1180F56D1ED
:1047F00009F00300D0BBAD4810380068C0F380005A
:1048000018B1E06808B9012053E7A84810380068DB
:1048100020F01900E1680843A44910390860FDF749
:1048200071F8054606E0FDF76DF8401B022801D936
:1048300003203EE79D4810380068C0F38000002840
:10484000F1D000BFFDF758F841F2030188421AD8B1
:10485000206940280BD195480C38006820F47C3042
:1048600040F4003091490C39086017E017E08F4898
:104870000C38006820F47C30216940EA01308B4913
:104880000C3908600AE089480C38006820F0FE40C6
:10489000217C40EA016085490C39086066E0E068E7
:1048A00088B382481038006820F01900E168084396
:1048B0007E4910390860FDF725F8054607E056E007
:1048C000FDF720F8401B022801D90320F1E67748C4
:1048D00010380068C0F380000028F1D000BFFDF759
:1048E0000BF841F2030188421AD8206940280BD105
:1048F0006E480C38006820F47C3040F400306B497E
:104900000C39086017E017E068480C38006820F49C
:104910007C30216940EA013064490C3908600AE0C2
:1049200062480C38006820F0FE40217C40EA0160BB
:104930005E490C39086019E05C481038006820F0C6
:1049400001005A4910390860FCF7DCFF054606E013
:10495000FCF7D8FF401B022801D90320A9E65348E1
:1049600010380068C0F380000028F1D100BF207823
:1049700000F0100010287CD14C48006800F0380886
:104980004A481830D0F80090B8F1080F06D0B8F1B6
:10499000180F3DD109F00300012839D143481038E0
:1049A0000068C0F3002020B1E069802801D0012018
:1049B0007FE600BFFCF7A0FF41F2030188421AD84E
:1049C000206A20280AD139480C38006820F0F840C5
:1049D00040F0804035490C39086018E033480C3805
:1049E000006820F0F84094F8201040EA81602F49D8
:1049F0000C3908600BE02D48001F006820F07C5047
:104A000094F8201040EA01602849091F086066E018
:104A1000E06978B325481038006840F080002349E9
:104A200010390860FCF76EFF054606E0FCF76AFFE8
:104A3000401B022801D903203BE61C4810380068BF
:104A4000C0F300200028F1D000BFFCF755FF41F271
:104A5000030188421CD8206A20280CD113480C3846
:104A6000006820F0F84040F0804010490C390860A0
:104A70001AE035E01CE00D480C38006820F0F840E2
:104A800094F8201040EA816008490C3908600BE076
:104A90000648001F006820F07C5094F8201040EA7F
:104AA00001600249091F086019E000001044025823
:104AB000FA48006820F08000F8490860FCF722FFFF
:104AC000054606E0FCF71EFF401B022801D9032023
:104AD000EFE5F2480068C0F300200028F2D100BFE3
:104AE000207800F00800082836D16069D0B1EB4882
:104AF0007430006840F00100E84974310860FCF748
:104B000001FF054606E0FCF7FDFE401B022801D927
:104B10000320CEE5E14874300068C0F3400000286F
:104B2000F1D019E0DD487430006820F00100DB4965
:104B300074310860FCF7E6FE054606E0FCF7E2FE8D
:104B4000401B022801D90320B3E5D4487430006823
:104B5000C0F340000028F1D1207800F02000202888
:104B600030D1A069B8B1CD48006840F48050CB493D
:104B70000860FCF7C7FE054606E0FCF7C3FE401BD5
:104B8000022801D9032094E5C4480068C0F34030EE
:104B90000028F2D016E0C148006820F48050BF49D8
:104BA0000860FCF7AFFE054606E0FCF7ABFE401BD5
:104BB000022801D903207CE5B8480068C0F34030E2
:104BC0000028F2D1207800F0040004287DD1B448F8
:104BD000006840F48070B2490860FCF793FE054617
:104BE00006E0FCF78FFE401B642801D9032060E536
:104BF000AB48006800F480700028F2D000BFA068C5
:104C0000012808D1A5487030006840F00100A34990
:104C1000703108602DE0A06868B9A0487030006865
:104C200020F001009D49703108600846006820F0BE
:104C3000040008601DE0A06805280DD19748703079
:104C4000006840F00400954970310860084600682B
:104C500040F0010008600CE090487030006820F0DF
:104C600001008E49703108600846006820F0040099
:104C7000086000BFA068A0B1FCF744FE054608E04C
:104C8000FCF740FE401B41F28831884201D90320E5
:104C90000FE5824870300068C0F340000028EFD074
:104CA00013E0FCF72FFE054608E0FCF72BFE401B47
:104CB00041F28831884201D90320FAE47748703004
:104CC0000068C0F340000028EFD1606A00287DD062
:104CD00072481030006800F03800182877D0606AF9
:104CE000022875D16D48006820F080706B4908601B
:104CF000FCF708FE054606E0FCF704FE401B022810
:104D000001D90320D5E465480068C0F3406000285D
:104D1000F2D100BFD4E90A1041EA00105F492831FE
:104D2000096840F2F332914308435C492831086036
:104D3000208E401EC0F30800616B491E4FF47E4276
:104D400002EA41210843218F491ED20102EA0141B2
:104D500008433C21095D491E120202EA0161084331
:104D60004E493031086000BF081F006820F0010084
:104D7000091F08604948343000684FF6F8718843CD
:104D8000A16C40EAC10045493431086043482C30E9
:104D9000006820F00C00216C084340492C31086069
:104DA0000846006820F00200616C08433B492C3142
:104DB00008600846006840F48030086008460068D3
:104DC00040F4003008600846006802E093E038E0F4
:104DD0001FE040F4802008600846006840F00100B1
:104DE00008602E48006840F080702C490860FCF78D
:104DF00089FD054606E0FCF785FD401B022801D928
:104E0000032056E425480068C0F340600028F2D033
:104E100071E02248006820F0807020490860FCF7AB
:104E200071FD054606E0FCF76DFD401B022801D927
:104E300003203EE419480068C0F340600028F2D126
:104E400059E0164828300768144830300668606A10
:104E5000012821D007F00301A06A81421CD1C7F3C9
:104E60000511E06A884217D1C6F30801206B401E85
:104E7000814211D1606B401EC6F3462188420BD19E
:104E8000A06B401EC6F30641884205D1E06B401E70
:104E9000C6F30661884205D001200AE400440258A6
:104EA0000048025815480068C0F3CC07A06CB8420F
:104EB00021D012480838006820F001000F49083955
:104EC0000860FCF71FFD054600BFFCF71BFD401BFB
:104ED000FBD00A4800684FF6F8718843A16C40EA9D
:104EE000C1000649086005480838006840F0010024
:104EF00002490839086000204AE40000344402589E
:104F000070B504462546681EB0F1807F01D30120AC
:104F10000FE0681E4FF0E02148610F214FF0FF3095
:104F200002F004FC00204FF0E021886107200861B6
:104F3000002070BD10B50346002200BF93F83C006E
:104F4000012801D1022010BD012083F83C0000BFE0
:104F500022F0FF00CC6840EA040222F440708C6822
:104F600040EA040222F480604C6840EA040222F421
:104F700000600C6840EA040222F480500C6940EAA8
:104F8000040222F400504C6940EA040222F48040FA
:104F90008C6A40EA040222F470200C8B40EA04423E
:104FA0000F4C1868A04203D00E4C1868A0420ED1D6
:104FB00022F470008C8C40EA045222F08070CC699C
:104FC00040EA040222F000700C6A40EA0402186809
:104FD000426400BF002083F83C0000BF00BFB2E77E
:104FE000000001400004014030B502460B4600BFFE
:104FF00092F83C00012801D1022030BD012082F846
:105000003C0000BF022082F83D0010684168106833
:105010008468214D1068A84203D0204D1068A84232
:1050200003D121F470015868014321F07001186820
:10503000014310684160184D1068A8421BD01068E9
:10504000B0F1804F17D0164D1068A84213D0154DFF
:105050001068A8420FD0144D1068A8420BD00F4D15
:105060001068A84207D0114D1068A84203D0104D17
:105070001068A84205D124F08004986804431068A1
:105080008460012082F83D0000BF002082F83C00CF
:1050900000BF00BFB1E70000000001400004014074
:1050A0000004004000080040000C004000180040D0
:1050B0000040014010B586B00446142101A8FBF75A
:1050C00072F93149206888421CD100BF2F4800681E
:1050D00040F010002D4908600846006800F01000FC
:1050E000009000BF00BF4FF4D44001900220029016
:1050F0000020039004900120059001A92448FCF7AA
:10510000F7FA3FE02349206888421BD100BF1F48BF
:10511000006840F004001D4908600846006800F07F
:105120000400009000BF00BFC02001900220029048
:105130000020039004900220059001A91648FCF776
:10514000D7FA1FE01549206888421BD100BF0F48DD
:10515000006840F008000D4908600846006800F04B
:105160000800009000BF00BF4FF4405001900220A3
:1051700002900020039004900220059001A90848A5
:10518000FCF7B6FA06B010BD00000140E04402583A
:1051900000100258000400400008025800080040B7
:1051A000000C02582DE9F04104460D461646002732
:1051B00000BF94F83C00012802D10220BDE8F08134
:1051C000012084F83C0000BF0C2E51D005DC4EB10C
:1051D000042E1ED0082E7AD133E0102E60D0142E6B
:1051E000F9D175E02946206801F04AFC2068806901
:1051F00040F00800216888612068806920F0040080
:10520000216888612068806929690843216888616C
:1052100078E02946206801F089FC2068806940F424
:105220000060216888612068806920F480602168BE
:10523000886120688069296940EA012021688861C5
:1052400060E02946206801F0CBFC2068C06940F08E
:1052500008002168C8612068C06920F00400216846
:10526000C8612068C069296908432168C86149E0AC
:105270002946206801F00EFD2068C06940F40060F6
:105280002168C8612068C06920F480602168C86115
:105290002068C069296940EA01202168C86131E0BD
:1052A0002946206801F030FD2068406D40F008007C
:1052B000216848652068406D20F004002168486539
:1052C0002068406D29690843216848651AE017E0A5
:1052D0002946206801F050FD2068406D40F40060D0
:1052E000216848652068406D20F480602168486529
:1052F0002068406D296940EA01202168486501E085
:10530000012700BF00BF00BF002084F83C0000BFA1
:10531000384653E710B504460CB9012010BD94F887
:105320003D0028B9002084F83C00204600F02AF80F
:10533000022084F83D00211D206801F033FB01208C
:1053400084F8480000BF84F83E0001213F20015549
:10535000402001554120015542200155432001556F
:1053600000BF00BF012084F84400452001554620BD
:1053700001554720015500BF012084F83D00002061
:10538000CCE7000008B51D4A016891420DD100BF6D
:105390001B49096841F00101194A11601146096869
:1053A00001F00101009100BF27E0164A0168914217
:1053B0000FD100BF12490839096841F00201104AB3
:1053C000083A11601146096801F00201009100BF1E
:1053D00013E00D4A016891420FD100BF0849083916
:1053E000096841F00401064A083A1160114609684B
:1053F00001F00401009100BF00BF08BD00000140A2
:10540000F04402580004004000080040014600BF7C
:1054100091F88400012801D102207047012081F811
:10542000840000BF2420C1F888000868026808686A
:10543000006820F001000B68186022F00052002084
:105440004866086802602020C1F8880000BF00207C
:1054500081F8840000BF00BFDFE770B504460D4649
:1054600000BF94F88400012801D1022070BD012002
:1054700084F8840000BF2420C4F8880020680668EF
:105480002068006820F001002168086020688068BA
:1054900020F06060284321688860204601F0A4FC69
:1054A000206806602020C4F8880000BF002084F82F
:1054B000840000BF00BFD9E770B504460D4600BFA9
:1054C00094F88400012801D1022070BD012084F8E5
:1054D000840000BF2420C4F8880020680668206883
:1054E000006820F00100216808602068806820F0D2
:1054F0006040284321688860204601F075FC2068E0
:1055000006602020C4F8880000BF002084F88400D2
:1055100000BF00BFD9E710B504460CB9012010BD8B
:10552000A06900B100E000BFD4F8880028B90020CD
:1055300084F88400204600F02BF82420C4F888006A
:105540002068006820F0010021680860A06A10B19E
:10555000204601F075FC204601F09AFD012800D19B
:10556000DDE72068406820F49040216848602068AA
:10557000806820F02A00216888602068006840F078
:10558000010021680860204601F0D6FCC7E7000052
:1055900010B5B8B00446142132A8FAF704FFC021B0
:1055A00002A8FAF700FF1E492068884235D102217F
:1055B0000020CDE90210209002A8FDF7D1FE08B12D
:1055C000FBF76DFB00BF1748006840F40030154939
:1055D00008600846006800F40030019000BF00BF7A
:1055E00000BF10480838006840F008000D4908392D
:1055F00008600846006800F00800019000BF00BF86
:1056000060203290022033900020349035900720A3
:10561000369032A90448FCF76BF838B010BD000092
:1056200000440040E8440258000C02582DE9F84FAD
:1056300004460E4617469946D4F88800202854D1CF
:1056400006B117B90120BDE8F88F00205434E0639B
:1056500021206063FCF756F9824627806780543C1E
:10566000A068B0F5805F04D1206910B90025B0466C
:1056700002E035464FF0000820E05346002280212A
:105680002046CDF8009001F0C9FF20B12020C4F8D9
:1056900088000320D7E745B9B8F80000C0F3080038
:1056A0002168886208F1020803E02878216888628E
:1056B0006D1CB4F85600401EA4F85600B4F856000D
:1056C0000028DAD15346002240212046CDF8009030
:1056D00001F0A4FF20B12020C4F888000320B2E725
:1056E0002020C4F888000020ADE70220ABE700BF0F
:1056F000FEE701688969C1F3400111B10021026828
:1057000091620168896901F0010129B9016889691B
:1057100041F0010102689161704700002DE9F74FE7
:1057200004460E4600272068D0F818800025DDF8D2
:10573000089008F01000102845D12168C86134E0B5
:10574000701C90B3FCF7DEF8A0EB0900B04200D863
:105750005EBB2068406800F4804A94F842B020683C
:105760008069C0F3C03070B1BAF5804F0BD0BBF187
:10577000200F08D02068406840F4804021684860CD
:10578000FCF7C0F8814609E0FCF7BCF8A0EB090083
:10579000192803D945F02005012705E02068806914
:1057A000C0F340100028EFD000BF20688069C0F32C
:1057B000401008B9002FC3D017B920202168C86154
:1057C00045F0040501272068D0F8188008F480709F
:1057D000B0F5807F06D145F001054FF48070216857
:1057E000C861012708F48060B0F5806F06D145F0EC
:1057F00008054FF480602168C861012708F4007033
:10580000B0F5007F06D145F002054FF40070216825
:10581000C8610127AFB12046FFF76BFF20684068E1
:105820000949084021684860606C28436064202072
:1058300084F84100002084F8420000BF84F8400052
:1058400000BF3846BDE8FE8F00E800FEF0B5059CBD
:10585000C1F309064FF47F0707EA02473E431E43A0
:10586000264326F00045066876684FF4806707EA0D
:10587000545767F0FC2747F4C047BE432E430768E0
:105880007E60F0BD2DE9F04104460D4617461E46E8
:10589000DDF818802BE0424631462046FFF73EFFF8
:1058A00010B10120BDE8F081701C00B3FCF72AF8AC
:1058B000A0EB0800B04200D8CEB92068806928402B
:1058C000A84201D1012000E00020B8420FD1606C55
:1058D00040F020006064202084F84100002084F81B
:1058E000420000BF84F8400000BF0120DAE72068D2
:1058F00080692840A84201D1012000E00020B84280
:10590000C9D00020CEE700002DE9F04104460E4644
:10591000174600254EE03A4631462046FFF7FEFE88
:1059200000B1012520688069C0F3401030B32DBB61
:1059300020688069C0F3800010B1208D00B100257F
:1059400020688069C0F30010C8B110202168C861C8
:105950000420606420202168C861206840681A49DA
:10596000084021684860202084F84100002084F825
:10597000420000BF84F8400000BF012501E0002084
:105980006064FBF7BFFFC01BB04200D896B98DB969
:1059900020688069C0F3800060B9606C40F020002E
:1059A0006064202084F8410000BF002084F840009B
:1059B00000BF012520688069C0F3800008B9002D70
:1059C000A9D02846BDE8F08100E800FE70B5044685
:1059D0000D46164622E0324629462046FFF79EFE37
:1059E00008B1012070BDFBF78DFF801BA84200D8D5
:1059F000A5B920688069C0F3401078B9606C40F0A8
:105A000020006064202084F84100002084F84200D7
:105A100000BF84F8400000BF0120E3E720688069F0
:105A2000C0F340100028D6D00020DBE770B5044654
:105A30000D46164624E0324629462046FFF76EFE04
:105A400008B1012070BD681CD0B1FBF75BFF801B63
:105A5000A84200D8A5B920688069C0F3400078B991
:105A6000606C40F020006064202084F84100002039
:105A700084F8420000BF84F8400000BF0120E1E745
:105A800020688069C0F340000028D4D00020D9E706
:105A9000FFB581B0044615461E464048047840488C
:105AA0000068012825D1002040EA4400C7B242F234
:105AB0001070012302AA394600903A48FCF7CAF850
:105AC00028B139A001F002FE012005B0F0BD01208F
:105AD00000EB4400C7B242F210702B463246394602
:105AE00000903048FCF704F810B134A001F0EEFD4E
:105AF00051E02B480068022824D1002040EA4400ED
:105B0000C7B242F21070012302AA39460090304811
:105B1000FCF7A0F820B124A001F0D8FD0120D4E7C3
:105B2000012000EB4400C7B242F210702B4632460F
:105B3000394600902648FBF7DBFF10B11FA001F0AB
:105B4000C5FD28E016480068032824D1002040EA5B
:105B50004400C7B242F21070012302AA39460090F5
:105B60001C48FCF777F820B10FA001F0AFFD012031
:105B7000ABE7012000EB4400C7B242F210702B46A5
:105B80003246394600901348FBF7B2FF10B10BA024
:105B900001F09CFD00BF00BF97E700003800002423
:105BA00044000024E80000242B2B777269746520E0
:105BB00062797465206661696C0D0A002D2D72652D
:105BC00061642062797465206661696C0D0A000069
:105BD0003C010024900100242DE9FF4105460E46BA
:105BE00014461F4629480578002040EA4500C5B202
:105BF00000200190029003908DF8046000BF04E043
:105C00003A5C411C01AB5A54401CA042F8DB2048CE
:105C10000068012811D142F21070631C01AA2946C4
:105C200000901C48FCF716F800282CD01AA001F0B0
:105C30004DFD012004B0BDE8F08115480068022840
:105C40000ED142F21070631C01AA29460090184838
:105C5000FCF700F8B8B110A001F038FD0120E9E729
:105C60000B48006803280ED142F21070631C01AA91
:105C7000294600900F48FBF7EDFF20B106A001F088
:105C800025FD0120D6E70020D4E7000038000024DD
:105C900044000024E80000242B2B777269746520EF
:105CA0006C656E2062797465206661696C0D0A000E
:105CB0003C0100249001002401468868C0F3C00024
:105CC00070470146886800F0010070470146886807
:105CD00000F00100704701468868C0F3007070470B
:105CE00001468868C0F38000704701468868C0F3A9
:105CF0008000704770B500F11404C1F3406504EBF7
:105D000085031C68C1F304560725B540AC43C1F3B5
:105D1000045502FA05F52C431C6070BD826822F020
:105D2000E0720A43826070472DE9FC4104460D464B
:105D30001646124908786B4606224321FFF7A8FE53
:105D40000746BFB99DF801009DF8001040EA012008
:105D500000B220809DF803009DF8021040EA012067
:105D600000B228809DF805009DF8041040EA01204B
:105D700000B230803846BDE8FC81000038000024C5
:105D800000B58BB00020089009900A901C2101A852
:105D9000FAF709FB1E481F490860002048600021EF
:105DA0001C488160C16004210161002101754175B9
:105DB000012181610021017741628162C162016339
:105DC000416380F83810FBF7C5FA08B1FAF767FFAE
:105DD0000020089008A90F48FAF764FF08B1FAF705
:105DE0005EFF0D48019006200290002003900B48B2
:105DF000049004200590002006908DF81D0001A954
:105E00000448FBF701F808B1FAF749FF0BB000BDF1
:105E100000200240840000240800900C0000FF478E
:105E200000B587B0142102A8FAF7BDFA00BF3948BF
:105E3000006840F01000374908600846006800F02C
:105E40001000019000BF00BF00BF0846006840F08E
:105E5000040008600846006800F00400019000BFDC
:105E600000BF00BF0846006840F080000860084698
:105E7000006800F08000019000BF00BF00BF08462E
:105E8000006840F0010008600846006800F001006A
:105E9000019000BF00BF00BF0846006840F002004C
:105EA00008600846006800F00200019000BF00BFD3
:105EB00000BF0846006840F0080008600846006817
:105EC00000F00800019000BF00BF002242F2020172
:105ED0001148FBF70BFD002208211048FBF706FDD7
:105EE00042F20200029001200390002004900590ED
:105EF00002A90948FBF7FCFB08200290012003904F
:105F000000200490059002A90448FBF7F1FB07B0BC
:105F100000BD0000E044025800080258000002588A
:105F200010B5134813490860134848600021114810
:105F300081600121C1600021016141618161C16114
:105F40000162FBF769FD08B1FAF7A9FE00210948D3
:105F5000FBF7DEFC08B1FAF7A2FE00210548FBF7CB
:105F60000CFD08B1FAF79BFE0120FBF73BFD10BDCD
:105F700000540040E80000244212400010B51348CD
:105F800013490860134848600021114881600121CD
:105F9000C1600021016141618161C1610162FBF762
:105FA0003BFD08B1FAF77BFE00210948FBF7B0FC86
:105FB00008B1FAF774FE00210548FBF7DEFC08B1D2
:105FC000FAF76DFE0220FBF70DFD10BD00580040F2
:105FD0003C0100244212400010B5134813490860E8
:105FE000134848600021114881600121C1600021EF
:105FF000016141618161C1610162FBF70DFD08B181
:10600000FAF74DFE00210948FBF782FC08B1FAF7C8
:1060100046FE00210548FBF7B0FC08B1FAF73FFE49
:106020000420FBF7DFFC10BD005C00409001002461
:106030004212400010B50B480B490860FF20486031
:106040000121094881600021C16001210161002115
:1060500041618161C1610162FCF7A8F808B1FAF7FA
:106060001EFE10BD00500052E401002400B595B0A2
:1060700000201290139014901C210BA8FAF793F9AA
:106080002C216846FAF78FF932483349086000201E
:1060900048600021304881604FF6FF71C1600021E7
:1060A000016141618161FFF735F908B1FAF7F7FD48
:1060B000002012901390149012A92748FEF794FF25
:1060C00008B1FAF7ECFD60200B9000200C900D90C9
:1060D0000E900F901090119000220BA91E48FFF710
:1060E00061F808B1FAF7DBFD04220BA91A48FFF7A3
:1060F00059F808B1FAF7D3FD08220BA91648FFF7A3
:1061000051F808B1FAF7CBFD0C220BA91248FFF7A2
:1061100049F808B1FAF7C3FD002000900190029001
:10612000039004904FF400500590002006900790D3
:106130004FF000700890002009900A9069460648C8
:10614000FEF7F8FE08B1FAF7AAFD0348FEF7B2FF22
:1061500015B000BD000001403002002400B58BB036
:106160000020089009900A901C2101A8FAF71BF959
:106170001B481C49086000204860002119488160C4
:106180004FF6FF71C160002101618161FFF7C2F824
:1061900008B1FAF784FD002008900A9008A9114878
:1061A000FEF722FF08B1FAF77AFD60200190002087
:1061B000029003900590002201A90A48FEF7F2FF21
:1061C00008B1FAF76CFD042201A90648FEF7EAFFC0
:1061D00008B1FAF764FD0348FEF76CFF0BB000BD91
:1061E000000400407C02002400B58BB00020089021
:1061F00009900A901C2101A8FAF7D5F81B481C4900
:106200000860002048600021194881604FF6FF7146
:10621000C160002101618161FFF77CF808B1FAF7E4
:106220003EFD002008900A9008A91148FEF7DCFE08
:1062300008B1FAF734FD602001900020029003902D
:106240000590002201A90A48FEF7ACFF08B1FAF751
:1062500026FD042201A90648FEF7A4FF08B1FAF7BB
:106260001EFD0348FEF726FF0BB000BD00080040EE
:10627000C802002410B51848184908604FF461207E
:106280004860002115488160C16001610C214161B5
:1062900000218161C1610162416200200F49886271
:1062A0000846FFF738F908B1FAF7F9FC00210B4866
:1062B000FFF702F908B1FAF7F2FC00210748FFF7EF
:1062C000CCF808B1FAF7EBFC0448FFF79FF808B1E7
:1062D000FAF7E5FC10BD0000004400401403002460
:1062E00000BFFEE700BFFEE770472DE9F04104461E
:1062F0000E4617469846069D12E0681C80B1FBF7D3
:1063000001FBA0EB0800A84200D84DB9042084F896
:106310004100606C40F0010060640120BDE8F08144
:1063200020688068304008B1012000E00020B842B9
:10633000E3D10020F2E700002DE9F04104460E46CB
:1063400000275548006800F00300032802D101200F
:10635000BDE8F08150482838006820F080604E4940
:1063600028390860FBF7CEFA054606E0FBF7CAFAC3
:10637000401B022801D90320EAE747482838006873
:10638000C0F3C0600028F1D100BF4348006820F48A
:106390007C30216840EA01303F490860A088401EF7
:1063A000C0F30800A168491E4FF47E4202EA412171
:1063B0000843A189491ED20102EA01410843217C18
:1063C000491E120202EA0161084333491031086094
:1063D00000BF3148001D006820F0C000616908431B
:1063E0002D49091D08600846006820F02000A169B9
:1063F00008432949091D08600846006820F010007C
:1064000008602548143000684FF6F8718843E16948
:1064100040EAC1002049143108601F48001D00688F
:1064200040F010001C49091D08602EB9084600689C
:1064300040F40020086012E0012E08D11648001D2B
:10644000006840F480101449091D086007E01248F4
:10645000001D006840F400100F49091D08600E4837
:106460002838006840F080600B4928390860FBF745
:1064700049FA054606E0FBF745FA401B022801D918
:10648000032065E7044828380068C0F3C06000288E
:10649000F1D038465CE70000284402582DE9F0416D
:1064A00004460E4600275548006800F00300032804
:1064B00002D10120BDE8F08150482838006820F062
:1064C00080504E4928390860FBF71CFA054606E063
:1064D000FBF718FA401B022801D90320EAE74748D6
:1064E00028380068C0F340700028F1D100BF43484D
:1064F000006820F07C70218840EA01503F49086024
:10650000A088401EC0F30800A168491E4FF47E42D7
:1065100002EA41210843A189491ED20102EA014150
:106520000843217C491E120202EA016108433349F3
:106530001831086000BF3148001D006820F4406039
:10654000616908432D49091D08600846006820F468
:106550000070A16908432949091D086008460068C0
:1065600020F48070086025481C3000684FF6F871F0
:106570008843E16940EAC10020491C3108601F4896
:10658000001D006840F480701C49091D08602EB988
:106590000846006840F48000086012E0012E08D12F
:1065A0001648001D006840F400001449091D0860E9
:1065B00007E01248001D006840F080700F49091D77
:1065C00008600E482838006840F080500B49283990
:1065D0000860FBF797F9054606E0FBF793F9401BC7
:1065E000022801D9032065E7044828380068C0F371
:1065F00040700028F1D038465CE70000284402587B
:10660000F0B52DED048B8DB004460D461646B7EE61
:10661000000AF0EE409A9FED670AB0EE408A9FEDC7
:10662000650AF0EE408A9FED630AB0EE409A06A834
:1066300008A907AB02AACDE9001009A90BA802F02E
:1066400043FA074627B101200DB0BDEC048BF0BD25
:10665000BDF8200000F4807000287CD09DED020A77
:10666000B8EEC00B9FED541B80EE012BB7EEC20BB2
:10667000F0EE409A9DED030AB8EEC00B9FED4E1B65
:1066800080EE012BB7EEC20BB0EE408A9DED040AFE
:10669000B8EEC00B9FED481B80EE012BB7EEC20B8E
:1066A000F0EE408A9DED050AB8EEC00B9FED421B4F
:1066B00080EE012BB7EEC20BB0EE409AB8EE001A96
:1066C00028EE011A21EE091AF0EE001A69EEA11A5D
:1066D00001EEA81AB7EEC11AB0EE410B01F03CF87A
:1066E000B7EEC00BB7EEC00A9FED351B20EE010BD5
:1066F000B7EEC00B84ED000AB8EE002A28EE022A9D
:1067000022EE082AF0EE002A68EEA22A02EEE82A1B
:10671000F7EE002A32EE222AB7EEC22AB0EE421B72
:10672000B0EE002A28EE822A22EE092AF0EE002A94
:1067300069EEA22A02EE882AB7EEC22AB0EE420B18
:1067400001F00EFAB7EEC00BB7EEC00A9FED1C1BAE
:1067500020EE010B00E02BE0B7EEC00B85ED000A48
:1067600029EEA92A08EE082A08EEE82A09EE492AA5
:10677000B7EEC22AB0EE421B28EE282A09EE892A7B
:10678000F0EE002A22EE222AB7EEC22AB0EE420B29
:1067900001F0E6F9B7EEC00BB7EEC00A9FED081B9B
:1067A00020EE010BB7EEC00B86ED000A00204BE790
:1067B000022049E700000000000000000000D04176
:1067C0006666666666A64C40704710B5FBF7F2FB3E
:1067D00010BD000000B59DB04C210AA8F9F7E3FDFB
:1067E000202102A8F9F7DFFD0220FBF7AFFC00BF74
:1067F000002001902A48006820F001002849086024
:106800000846006800F0010001902648006840F446
:106810004040244908600846006800F44040019068
:1068200000BF00BF00BF1F48006800F40050B0F573
:10683000005FF8D102200A9001200D9040200E90B8
:1068400002201390002114910421159132211691F8
:1068500002211791189119910C211A9100211B9175
:106860001C910AA8FDF720FF08B1FAF718FA3F209B
:1068700002900320039000200490082005904020FF
:10688000069007900001089040200990022102A87C
:10689000FDF71AFC08B1FAF702FA1DB000BD0000BE
:1068A0002C040058184802583448006840F470001E
:1068B000324908603248006800F00F00072806D20D
:1068C0002F48006820F00F00C01D2D4908602D489A
:1068D000006840F001002B49086000202949103170
:1068E000086028480068284908402649086024486C
:1068F000006800F00F00072806D92148006820F042
:106900000F00C01D1E49086000201E491831086094
:10691000091D0860091D08601C481A4928310860D3
:106920001B48091D08601B48091D08600020091D3F
:1069300008601848091D08600020091D08601548F6
:10694000091D08600020091D08600E48006820F439
:1069500080200C49086000200A49603108600E4818
:1069600000686FF30F00B0F1005F02D201200B4905
:10697000086043F2D2000A490860704788ED00E0E1
:1069800000200052004402587FEDF6EA00020202A5
:106990000000FF01800201010010005C088100512D
:1069A0000040005210B502682D4B98420ED0B0F155
:1069B000804F0BD02B4B984208D02B4B984205D0E0
:1069C0002A4B984202D02A4B984203D122F07002FF
:1069D0004B681A43224B984217D0B0F1804F14D025
:1069E000204B984211D0204B98420ED01F4B98421A
:1069F0000BD01F4B984208D01E4B984205D01E4B1F
:106A0000984202D01D4B984203D122F44072CB68C9
:106A10001A4322F080034C6943EA040202608B6847
:106A2000C3620B6883620E4B98420BD0104B9842A6
:106A300008D0104B984205D00F4B984202D00F4B14
:106A4000984201D10B69036301234361036903F099
:106A500001031BB1036923F00103036110BD0000B2
:106A6000000001400004004000080040000C00400D
:106A70000004014000400140004401400048014042
:106A800030B5026A056A25F001050562436884692C
:106A9000204D2C4024F003040D682C4322F0020208
:106AA0008D682A431C4DA84200D10FE01B4DA8421F
:106AB00000D10BE01A4DA84200D107E0194DA842C1
:106AC00000D103E0184DA84206D100BF22F0080211
:106AD000CD682A4322F004020F4DA8420BD00F4D7F
:106AE000A84208D00E4DA84205D00E4DA84202D0B3
:106AF0000D4DA84207D123F4807323F400734D6930
:106B00002B438D692B43436084614D68456302626A
:106B100030BD00008FFFFEFF000001400004014077
:106B200000400140004401400048014030B5026A85
:106B3000056A25F01005056243688469224D2C40E2
:106B400024F440740D6844EA052422F020028D6884
:106B500042EA05121D4DA84200D10FE01C4DA8428B
:106B600000D10BE01B4DA84200D100BF1A4DA84236
:106B700000D100BF194DA84207D106E022F08002E3
:106B8000CD6842EA051222F04002104DA8420BD017
:106B90000F4DA84208D00F4DA84205D00E4DA84277
:106BA00002D00E4DA84209D123F4806323F4006380
:106BB0004D6943EA85038D6943EA85034360846137
:106BC0004D688563026230BDFF8FFFFE000001400B
:106BD00000040140004001400044014000480140E1
:106BE00030B5026A056A25F4807505624368C46998
:106BF000224D2C4024F003040D682C4322F4007233
:106C00008D6842EA05221E4DA84200D10FE01D4DBD
:106C1000A84200D10BE01C4DA84200D100BF1B4D83
:106C2000A84200D100BF1A4DA84207D106E022F4C5
:106C30000062CD6842EA052222F48062104DA8422B
:106C40000BD0104DA84208D00F4DA84205D00F4DD3
:106C5000A84202D00E4DA84209D123F4805323F458
:106C600000534D6943EA05138D6943EA05134360F8
:106C7000C4614D68C563026230BD00008FFFFEFF36
:106C80000000014000040140004001400044014078
:106C90000048014030B5036A056A25F48055056255
:106CA0004468C269124D2A4022F440720D6842EADB
:106CB000052223F400538D6843EA05330D4DA842A5
:106CC0000BD00D4DA84208D00C4DA84205D00C4D5C
:106CD000A84202D00B4DA84204D124F480444D694F
:106CE00044EA85144460C2614D680564036230BDA6
:106CF000FF8FFFFE00000140000401400040014002
:106D0000004401400048014030B5026A056A25F49C
:106D1000803505624368446D114D2C400D682C434D
:106D200022F400320D8942EA05420E4DA8420BD0F2
:106D30000D4DA84208D00D4DA84205D00C4DA842DB
:106D400002D00C4DA84204D123F480334D6943EAAC
:106D50000523436044654D688565026230BD0000CF
:106D60008FFFFEFF00000140000401400040014091
:106D7000004401400048014030B5026A056A25F42C
:106D8000801505624368446D114D2C400D6844EA3E
:106D9000052422F400120D8942EA05520D4DA84245
:106DA0000BD00D4DA84208D00C4DA84205D00C4D7B
:106DB000A84202D00B4DA84204D123F480234D6990
:106DC00043EA8523436044654D68C565026230BD72
:106DD000FF8FFFFE00000140000401400040014021
:106DE000004401400048014070B5456E2DB90125B1
:106DF000A0F86A50A0F868501CE010231024056821
:106E0000AD68C5F342610568AD686A0F0A4DAD5CB7
:106E100015FB04F5094EB65C95FBF6F5A0F86A5033
:106E2000054D6D5C15FB03F5044E765C95FBF6F5A0
:106E3000A0F8685070BD0000F6BC0008FEBC000859
:106E400090F8281001F00801082907D10168496865
:106E500021F40041826B11430268516090F82810C0
:106E600001F0010139B10168496821F40031C26AB9
:106E700011430268516090F8281001F002010229C4
:106E800007D10168496821F48031026B114302681F
:106E9000516090F8281001F00401042907D101681D
:106EA000496821F48021426B11430268516090F8D7
:106EB000281001F01001102907D10168896821F418
:106EC0008051C26B11430268916090F8281001F064
:106ED0002001202907D10168896821F40051026C42
:106EE00011430268916090F8281001F04001402998
:106EF00013D10168496821F48011426C1143026882
:106F00005160416CB1F5801F07D10168496821F4D7
:106F1000C001826C11430268516090F8281001F0A2
:106F20008001802907D10168496821F40021C26CE1
:106F3000114302685160704738B504460020C4F818
:106F40009000FAF7DFFC05462068006800F00800B2
:106F5000082821D16FF07E402B4600224FF400110B
:106F60000090204600F05AFBB0B100BF00BF21687E
:106F700051E8001F21F08000226842E8000100294A
:106F8000F5D100BF2020C4F8880000BF002084F89D
:106F9000840000BF032038BD2068006800F00400B2
:106FA000042830D16FF07E402B4600224FF4800140
:106FB0000090204600F032FB28B300BF00BF2168DC
:106FC00051E8001F21F49070226842E80001002976
:106FD000F5D100BF00BF00BF2168083151E8001F94
:106FE00021F001002168083141E80002002AF3D1B4
:106FF00000BF2020C4F88C0000BF002084F884006B
:1070000000BF0320C7E72020C4F88800C4F88C0024
:107010000020E066206700BF84F8840000BF00BF46
:10702000B9E7000000BF00BF026852E8002F22F459
:107030009071036843E80012002AF5D100BF00BF39
:1070400000BF0268083252E8002F104B02EA030129
:107050000268083242E80013002BF2D100BFC16E73
:1070600001290CD100BF00BF026852E8002F22F0B6
:107070001001036843E80012002AF5D100BF202167
:10708000C0F88C100021C16641677047FEFFFFEF1A
:107090002DE9F04F89B0054600200890F84928688E
:1070A000884200D100E000BF2969A86808436969E7
:1070B0000843E96940EA010828680068F149084086
:1070C00040EA0800296808602868406820F44050B9
:1070D000E968084329684860D5F81880E8492868B5
:1070E000884202D0286A40EA080828688068E64991
:1070F000084040EA0800296888602868C06A20F0D3
:107100000F00696A08432968C86200BFDF49286820
:10711000884220D1DE48006800F03800182811D0DD
:1071200005DC48B1082809D0102811D108E0202832
:107130000AD028280CD109E001240BE0042409E03E
:10714000082407E0102405E0202403E0402401E0A7
:10715000802400BFF8E0CF492868884219D1CC4884
:10716000006800F00700062810D2DFE800F00305F1
:1071700007090B0D00240BE0042409E0082407E0B4
:10718000102405E0202403E0402401E0802400BF17
:10719000DAE0C1492868884219D1BD48006800F08A
:1071A0000700062810D2DFE800F0030507090B0DE1
:1071B00000240BE0042409E0082407E0102405E083
:1071C000202403E0402401E0802400BFBCE0B34958
:1071D0002868884219D1AE48006800F007000628E8
:1071E00010D2DFE800F0030507090B0D00240BE0C7
:1071F000042409E0082407E0102405E0202403E02B
:10720000402401E0802400BF9EE0A5492868884210
:1072100019D19F48006800F00700062810D2DFE867
:1072200000F0030507090B0D00240BE0042409E01E
:10723000082407E0102405E0202403E0402401E0B6
:10724000802400BF80E097492868884220D1904878
:10725000006800F03800182811D005DC48B1082873
:1072600009D0102811D108E020280AD028280CD1F4
:1072700009E001240BE0042409E0082407E01024BD
:1072800005E0202403E0402401E0802400BF5BE00F
:1072900085492868884219D17D48006800F00700B8
:1072A000062810D2DFE800F0030507090B0D0024C3
:1072B0000BE0042409E0082407E0102405E0202462
:1072C00003E0402401E0802400BF3DE077492868C6
:1072D000884219D16E48006800F00700062810D2D5
:1072E000DFE800F0030507090B0D00240BE0042480
:1072F00009E0082407E0102405E0202403E04024EE
:1073000001E0802400BF1FE05D49286888421AD14F
:107310005F48001D006800F00700062810D2DFE873
:1073200000F0030507090B0D02240BE0042409E01B
:10733000082407E0102405E0202403E0402401E0B5
:10734000802400BF00E0802400BF4D4928688842A7
:107350007DD1102C1AD006DC022C09D0042C0BD0C5
:10736000082C29D10DE0202C21D0402C24D120E064
:10737000FBF744F8064623E005A8FBF769F9069EEB
:107380001EE002A8FBF77CFA039E19E0404854383F
:107390000068C0F3401040B13D4854380068C0F365
:1073A000C101434820FA01F600E0414E08E0414E99
:1073B00006E04FF4004603E000260120089000BFDD
:1073C00000BF002E10D03C49686A31F81000B6FBAF
:1073D000F0F9686800EB4000484503D8686800038E
:1073E000484502D20120089003E13349686A31F828
:1073F00010C06246002330461946F8F76BFF4FF481
:10740000807300228446ACFB030B01FB03B10CFB31
:10741000021C69684908034659184CEB0200CDE983
:107420000010D5F804C06246002308460199F8F719
:1074300051FF0746B7F5407F06D3B7F5801F03D24B
:107440002868C760D5E002E001200890D1E0E86933
:10745000B0F5004F7BD1082C39D005DC5CB1012C94
:107460002CD0042C4CD12DE0102C35D0202C42D027
:10747000402C45D141E0FCF7DDFF064644E000002A
:10748000000C0058F369FFCFFFF4FF11001001401A
:10749000544402580044004000480040004C004062
:1074A000005000400014014000780040007C004083
:1074B0000090D00300093D00DEBC0008FCF7CCFFC3
:1074C000064621E005A8FBF7C3F8069E1CE002A8CB
:1074D000FBF7D6F9039E17E04C480068C0F3401054
:1074E00038B14A480068C0F3C101494820FA01F6A2
:1074F00000E0474E08E0474E06E04FF4004603E048
:1075000000260120089000BF00BFFEB14249686A12
:1075100031F81000B6FBF0F04000696800EB510054
:10752000B0FBF1F7102F0FD3B7F5803F0CD24FF619
:10753000F07007EA000AC7F342004AEA000A286826
:10754000C0F80CA055E002E00120089051E0082CA2
:107550001AD005DC5CB1012C0DD0042C2DD10EE02D
:10756000102C16D0202C23D0402C26D122E0FCF762
:1075700061FF064625E0FCF76FFF064621E005A8FF
:10758000FBF766F8069E1CE002A8FBF779F9039E5C
:1075900017E01E480068C0F3401038B11B4800686F
:1075A000C0F3C1011A4820FA01F600E0184E08E0C5
:1075B000184E06E04FF4004603E000260120089034
:1075C00000BF00BFAEB11449686A31F81000B6FBC5
:1075D000F0F0696800EB5100B0FBF1F7102F06D313
:1075E000B7F5803F03D2B8B22968C86001E0012036
:1075F00008900120A5F86A00A5F8680000206867D7
:10760000A867089809B0BDE8F08F00000044025850
:107610000090D00300093D00DEBC00082DE9F041D8
:1076200004460D4617469846069E41E0701C002809
:107630003ED0FAF767F9A0EB0800B04200D816B9BF
:107640000320BDE8F0812068006800F0040070B3FA
:10765000802D2DD0402D2BD02068C069C0F3C000F4
:1076600078B10820216808622046FFF7DBFC08207B
:10767000C4F8900000BF002084F8840000BF0120FF
:10768000DFE72068C069C0F3C02080B14FF400601C
:10769000216808622046FFF7C5FC2020C4F890004E
:1076A00000BF002084F8840000BF0320C9E7FFE783
:1076B0002068C0692840A84201D1012000E00020D4
:1076C000B842B3D00020BCE700BFFEE70FB4054BC3
:1076D00010B503A9044A029800F056FC10BC5DF8EE
:1076E00014FB0000B59300085C00002403B401986B
:1076F0004100009850EAC12018BF04204A0D18BF6D
:1077000040F0010040F2FF72B2EB515F08BF40F061
:107710000200012808BF052002B070470248006837
:10772000C0F30220704700000CED00E010B5002807
:1077300004DB0A07130E054A135406E00A07140E69
:10774000034A00F00F031B1FD45410BD00E400E0F7
:1077500018ED00E00000000070B56B482DED020B45
:107760002DED0A8B82B00D9D25F000449FED68BB86
:107770009FED699B84422EDBA4F140510C98A1F14E
:107780007F6108430FD06648844202DC18D10C9810
:10779000B0B19DED0C0B02B0BDEC0A8B02B0BDE8A0
:1077A000704000F0F9BA9DED0C0B9DED0C1B20EE26
:1077B0000B0B01EE090B02B0BDEC0A8B02B070BDE1
:1077C000012000F019FB02B0BDEC0A8B02B0BDE84D
:1077D000704000F0E9BA53489FED538B844230DA91
:1077E0009DED0C0BB4F1795F0ADA51EC100BFFF749
:1077F0007DFF042808BF00F0E3FA9DED0C0BDAE7EB
:1078000020EE009B4A480621B0EE490B784400F078
:107810008BFA20EE09AB4748B0EE490B04217844BF
:1078200000F082FA09EE008B8AEE080B8DED000B5A
:107830009DED0C0B9DED0C1B9DED002B01EE020B45
:10784000B9E79DED0C0B51EC100B01F0A7FD41ECDD
:10785000100B9FED391B3A4838EE400B06218DED99
:10786000000B20EE01ABB0EE4A0B784400F05CFA5E
:1078700020EE0ACB3348B0EE4A0B0421784400F0E6
:1078800053FA0AEE008B51EC1A0B03F0CDFB41ECDE
:10789000110B2D489FED2E2BA0420EDC8CEE080B19
:1078A0008DED000B9DED003BB0EE410B01EE030BA7
:1078B00010EE029B3BEE490B21E08DED001B0020FA
:1078C00000909DED000B9DED003B00EE43AB31EED3
:1078D000000B21EE021B8AEE003B8CEE080B03EE40
:1078E000429B9DED003B11EE009B9FED1B1BB0EEFC
:1078F000410B03EE420B39EE400B31EE400B002DF5
:10790000D8BFB1EE400B56E70000F03F000000008A
:10791000182D4454FB21F93F075C143326A6913CF3
:107920000000F07F0000E03F000000000000F03F9A
:107930000845000026450000000000000000E03F70
:10794000AA440000C84400003333EF3F00000000A9
:107950000000000000000040182D4454FB21E93FC6
:1079600070B565482DED020B2DED048B059D25F0BE
:107970000044A04218DC6148844202DC0AD1049829
:1079800040B19DED040BBDEC048B02B0BDE870402E
:1079900000F002BA002DCCBF9FED590B9FED5A0BA2
:1079A000BDEC048B02B070BD5948A04215DD5948AA
:1079B000A042D8BF4FF0FF3455DD9DED040B51ECD4
:1079C000100BFFF793FE042808BF00F0F9F99DEDB6
:1079D000040BBDEC048B02B070BD9DED040B51ECAB
:1079E000100B01F0DBFCCDE904014B489FED4C0B83
:1079F000A0421CDD4C48A0420BDD9DED042B002471
:107A00009FED4B1B12EE010B32EE011B80EE012BA2
:107A100027E09DED041B9DED042B012431EE401B5E
:107A200032EE000B81EE002B8DED042B1BE0424863
:107A3000A0420FDD9DED042B02249FED411B9DED27
:107A4000043B32EE412B03EE010B82EE001B8DED69
:107A5000041B08E09DED040B9FED3B1B032481EE0E
:107A6000002B8DED042B9DED040B3948062120EEF3
:107A7000009B29EE098BB0EE480B784400F054F9D6
:107A800020EE099B3348B0EE480B0521784400F006
:107A90004BF920EE080B002C0BDA9DED042B39EE90
:107AA000001B9DED040BBDEC048B02B002EE410BFC
:107AB00070BD2948784439EE000B00EBC4009DED01
:107AC000042B90ED001B254812EE001B9DED040BCE
:107AD00031EE400B784400EBC400002D90ED001B0C
:107AE00031EE400BB8BFB1EE400BBDEC048B02B0E1
:107AF00070BD000000000000000010440000F07F96
:107B0000182D4454FB21F93F182D4454FB21F9BF93
:107B10000000DC3F0000203E0000F33F00000000BA
:107B2000000000000000F03F0000E63F0000000001
:107B30000000000000000040008003400000000042
:107B4000000000000000F83F000000000000F0BF4F
:107B50005243000018430000D04200009042000051
:107B600070B5614E2DED040B2DED048B82B0DDF868
:107B700024C0DDE907235C422CF000411C4341EAAC
:107B8000D474069D22F00040B44205D86C422C43C8
:107B900040EAD474B4420BD99DED081B9DED060B51
:107BA00002B0BDEC048B04B0BDE8704000F0F7B843
:107BB000ACF14054A4F17F641C430BD0022404EACE
:107BC000AC7444EAD27405439FED498B9FED4A2B78
:107BD0000DD016E09DED060B51EC100B00F0B8FD3A
:107BE00041EC100B02B0BDEC048B04B070BD002C56
:107BF00014BF012C9DED060BF4D0022C2ED0032CCB
:107C00002FD00B439FED3E1B9FED3F0B0AD0B1429F
:107C10001DD1B04209D121F0804120F0804009916E
:107C2000079014E0002ADDDA15E0394B7B44002C84
:107C300008BF93ED000BD5D0012C04BF93ED000BD2
:107C4000B1EE400BCED0022C08D0032C09D0B042AC
:107C50000AD1002AC6DAB0EE410BC3E7B0EE480BFA
:107C6000C0E7B0EE420BBDE7401A00159FED2A9B1E
:107C70003C28C8BF8DED000B15DCBCF1000FBCBF6C
:107C800010F13C0F8DED009B0DDB9DED061B9DED76
:107C9000082B81EE020B51EC100B01F07FFB00F082
:107CA00057FDCDE9000194B1012C0CD09DED001BD6
:107CB0009FED1B0B022C31EE400B0CBF38EE400B3E
:107CC00030EE480B8EE7019880F0004001909DED6A
:107CD000000BB4EE490BF1EE10FA04BF022000F0E5
:107CE0008BF89DED000B7DE70000F07F00000000A9
:107CF000182D4454FB210940182D4454FB2109C080
:107D0000182D4454FB21F9BF182D4454FB21F93F91
:107D1000D041000000000000000000000000000052
:107D2000075C143326A6A13C491E00EBC102B0EE4D
:107D3000401B92ED000B31F006020DD0491E00EB06
:107D4000C102B0EE403B92ED002B31F00602B0EEE6
:107D5000420B03EE010BF1D1022914D004290AD001
:107D6000062918BF704790ED0A2B00EE012B90ED0D
:107D7000080B02EE010B90ED062B00EE012B90EDAF
:107D8000040B02EE010B90ED022B00EE012B90EDA7
:107D9000000B02EE010B704730EE000B704730EE27
:107DA000010B7047000000009FED031B81EE010BEB
:107DB000704700000000000000000000000000000C
:107DC0009FED030B20EE000B704700000000000049
:107DD000000000000000001002E008C8121F08C1E7
:107DE000002AFAD170477047002001E001C1121F3C
:107DF000002AFBD17047000001490860704700006D
:107E0000600000242DE9FF5F82B00021DDE904302D
:107E1000020DDDF840B0034318D044F61050A2F232
:107E2000FF3242431514119801281FD0A5EB0B0017
:107E3000401C5FEA000A4FF000064E4FDFF8389111
:107E4000B046504615D5CAF1000413E0119801243C
:107E50004AA3012801D16FEA0B010298119AC0E9E7
:107E60000031C0E9024206B0BDE8F09FCBF100004E
:107E7000DFE704460021404A491842EB0450CDE9AF
:107E8000001012E0E00707D032463B464046494624
:107E9000F8F77DFB8046894632463B461046194638
:107EA000F8F775FB06460F466410002CEAD1DDE9B1
:107EB0000401DDE90023BAF1000F06DAF8F767FBE9
:107EC00042464B46F8F763FB05E0F8F7D2FB424623
:107ED0004B46F8F7CEFB04460E460022284BF8F737
:107EE0004FFC03D84FF0FF30014607E00022254B3E
:107EF00020463146F8F7A4FAF8F72AFC102409E0E6
:107F0000002C0ADB0A220023F8F7E4F9039B303245
:107F10001A55641E50EA0102F2D1641C039AC4F19E
:107F200011031444119A012A03D0012208430DD1F0
:107F30000AE0084304D000204FF0110B119072E7C3
:107F4000A3EB0B056D1E0DE05B4504DD4FF0000259
:107F500005F1010504E003DA4FF00002A5F1010587
:107F6000002AECD002981199C0E90231C0E900451D
:107F700079E70000000014400000F03F30000000EE
:107F80000000F0430000E03F2DE9FF4F95B09A4616
:107F9000884606460025EEE1252877D100242746AD
:107FA000F94A0121039400E0044316F8013F203B05
:107FB00001FA03F01042F7D130782A2811D06FF07F
:107FC0002F033078A0F13002092A16D8039A44F022
:107FD000020402EB820203EB42021044761C03907F
:107FE000EFE758F8042B0392002A03DA504244F4D6
:107FF0000054039044F00204761C30782E2816D1E9
:1080000016F8010F44F004042A280DD06FF02F0257
:108010003078A0F13003092B09D807EB870302EB76
:108020004303C718761CF3E758F8047B761C3078B6
:108030006C280FD006DC4C2817D068280DD06A2891
:1080400014D104E0742810D07A280FD10DE044F444
:1080500000140AE044F4801401E044F440147278FF
:10806000824202D104F58014761C761C3078662892
:108070000BD013DC582877D009DC002875D04528B0
:10808000F6D04628F4D047281AD193E118E06328A7
:1080900035D0642879D0652812D18BE1702873D04F
:1080A00008DC6728F1D069286FD06E280DD06F28C2
:1080B00006D1ACE073282CD0752874D0782853D022
:1080C0005246179990476D1C54E1C4F302500228A0
:1080D00009D003280DD0D8F8001004280DD00D6069
:1080E00008F1040846E1D8F80010EA17C1E9005287
:1080F000F6E7D8F800100D80F2E70D70F0E718F8F9
:10810000041B8DF8001000208DF80100EB460120C3
:1081100003E058F804BB4FF0FF3061074FF0000157
:1081200002D40DE009F101018946B9420FDA814517
:10813000F8DB1BF809100029F4D108E009F101016E
:1081400089468142FADB1BF809100029F6D1039811
:108150005346A0EB090721463846179A00F080FAEB
:10816000284400EB090507E044E008E10DE01BF8B6
:10817000010B524617999047B9F10109F7D25346BE
:1081800021463846179AF2E039E00A21C4F3025238
:108190004FF0000B0091022A06D058F8040BC117CB
:1081A000032A09D00AE023E008F1070020F00702C3
:1081B000F2E80201904605E000B2C117042A01D19D
:1081C00040B2C117002906DA0A460021404261EB9D
:1081D00002012D2202E0220504D52B228DF8042075
:1081E000012203E0E20701D02022F7E7914657E0A1
:1081F0000A2100E010214FF0000B00910BE010214C
:108200004FF0000B44F004040827009103E008201D
:108210004FF0000B0090C4F30252022A05D058F828
:10822000040B0021032A08D008E008F1070020F021
:108230000702F2E80201904603E080B2042A00D16E
:10824000C0B24FF0000922072AD53278702A07D031
:10825000DDF800C08CF0100C5CEA0B0C05D00EE0D1
:1082600040228DF80420012208E050EA010306D0E4
:1082700030238DF804308DF8052002229146009BB2
:1082800083F0080353EA0B030AD150EA010201D13B
:10829000620705D530228DF804204FF001097F1EBA
:1082A0003278582A04D039A20C920CAA02920BE020
:1082B0003BA2F9E75B46009AF8F70CF80C9B9B5C35
:1082C000029A521E0292137050EA0102F2D10298F1
:1082D00004A9081A00F1200B600702D524F48034A9
:1082E00000E001275F4502DDA7EB0B0000E0002066
:1082F00000EB0B01009003984944401A0390E003FF
:1083000006D453462146179A039800F0A9F905446C
:10831000002706E001A85246C05D179990476D1CE2
:108320007F1C4F45F6DBE0030CD553462146179AD8
:10833000039800F095F9054404E03020524617995F
:1083400090476D1C0099481E00900029F5DC08E05C
:108350000298029952460078491C02911799904759
:108360006D1CBBF10001ABF1010BF1DC5BE100F036
:1083700065F90544761C307800287FF40DAE19B0FD
:108380002846BDE8F08F0000092801003031323363
:108390003435363738396162636465660000000041
:1083A000303132333435363738394142434445462B
:1083B00000000000600700D4062708F1070020F045
:1083C0000700F0E80223804603F0004C5FEA0C004F
:1083D00001D097A009E0200501D596A005E0E007AF
:1083E00001D095A001E0AFF24C001390307823F05B
:1083F000004365280CD006DC452809D046281DD04E
:1084000047287FD13BE0662818D067287AD136E02C
:108410000021112F01DB112000E0781CCDE90001C3
:1084200004A90CA8FFF7EEFCDDE90D010C9A4FF052
:10843000000B07F10109109200914EE04FF000404F
:108440000097CDE9011004A90CA8FFF7DBFCDDE9DA
:108450000D020C9B0F994FF0000B91461093009268
:1084600011B9791C00EB0109B7EB090003D4C0F185
:10847000FF3B07F10109A9EB0700019042E0012F42
:1084800000DA01270021112F01DD112000E038461C
:10849000CDE9000104A90CA8FFF7B4FCDDE90D014A
:1084A0000C9A00914FF0000BB946109221070FD49F
:1084B000009A4A4503DA914601E0A9F10109B9F1B0
:1084C000010F05DD109AA9F10101515C3029F4D0AA
:1084D000B84202DA10F1040F03DA0121CDE90110EC
:1084E00010E0002803DC8344A9EB000102E0411CFA
:1084F000494500DD8946A0EB0B00401C01904FF080
:1085000000400290200705D40198484502DB4FF057
:10851000FF30019000208DF84B0002980DF14B07C1
:10852000B0F1004F25D002200C902B200D90029826
:1085300000280CDA404202902D200D9007E00A211D
:108540000298F7F748FF3031029007F8011D0C99A7
:10855000481E0C900029F2DC02980028EFD1791E09
:108560000D980870307800F0200040F0450007F8C2
:10857000020D11A8C01BC01D02901398007800B115
:10858000012000EB0901019801EBE0710298014420
:108590000398401A401E0390E00306D45346214638
:1085A000179A039800F05CF805441398007818B106
:1085B0005246179990476D1CE00323D55346214638
:1085C000179A039800F04CF805441BE0BBF1000F2C
:1085D00007DB0098584504DD1098179910F80B0038
:1085E00001E0179930205246904701980BF1010B9A
:1085F000401E05F10105019004D12E205246179925
:1086000090476D1CB9F10001A9F10109DEDC05E01C
:1086100017F8010B5246179990476D1C0299481E96
:1086200002900029F4DC53462146179A03989EE6EF
:108630002D0000002B000000200000002DE9F0417B
:10864000044600251E461746880404D405E0394632
:108650002020B0476D1C641EF9D52846BDE8F08186
:108660002DE9F041044600251E469046C80301D579
:10867000302700E02027880404D505E0414638462D
:10868000B0476D1C641EF9D52846BDE8F081000096
:10869000F0B52DED028B83B006460F4600256846E7
:1086A00000F096FE002448E056F8241057F82420E5
:1086B000881A002801DB014600E0414200EE101A52
:1086C000B8EEC00ADFED200A80EE208A684600EB93
:1086D000840090ED000AB5EEC00AF1EE10FA19D050
:1086E000684600EB8400D0ED000A88EE200AF7EE21
:1086F000000A70EE608A00BFB0EEE80A1348D0EDC1
:10870000090AB4EEE00AF1EE10FA15DD0120A040EE
:10871000054311E00D4890ED070AB4EEC80AF1EEEA
:1087200010FA06DC90ED080AB4EEC80AF1EE10FA71
:1087300002D20120A0400543641C032CB4DB284670
:1087400003B0BDEC028BF0BD00008047C0B0000854
:1087500010B541EC100BFFF703F951EC100B10BDF5
:108760002DE9F0410446E07800F0C006E07800F022
:108770003F05607800F0010098B1EF102846E91736
:1087800005EB5171C910A5EBC101491C01F0FF08AF
:108790000B48006820B10A484146026838469047B5
:1087A00000BF607800F0080030B10548406818B19B
:1087B000B011034A516888470020BDE8F0810000ED
:1087C0006400002438B5044664B120208DF8000010
:1087D00028208DF8010030208DF8020038208DF817
:1087E000030004E0A32204216846F7F7D5FD6A469A
:1087F000042140F69E2002F089FA01F073FE38BD94
:108800003EB5044602208DF80000CA208DF8010014
:10881000E3208DF8020009208DF803006A46042148
:10882000682002F073FAA3208DF8000004F04000E5
:1088300048B1C0208DF80100C8208DF80200C22088
:108840008DF8030006E0A3208DF801008DF80200EA
:108850008DF8030004F4C07048B1C4208DF8040002
:10886000CC208DF80500C6208DF8060006E0A32078
:108870008DF804008DF805008DF80600A3208DF812
:1088800007008DF808008DF809006A460A2140F6B5
:10889000A72002F03BFA04F0030018B120208DF865
:1088A000000002E0D8208DF800006A46012140F661
:1088B000B62002F02BFA04F0200018B1012000F0DD
:1088C000ADF802E0002000F0A9F804F4C07008B38D
:1088D00004F4807060B1B2208DF800008B208DF818
:1088E0000100B6208DF802009B208DF803000BE0FC
:1088F000B0208DF8000080208DF80100B4208DF8A4
:10890000020090208DF803006A46042140F6A22060
:1089100002F0FCF904F0010020B3F8208DF800000B
:108920006A4601214FF40B6002F0F0F9FA210720AA
:1089300000F02EFC072000F0F5FB012000F015FCF4
:10894000642000F005FD4FF4FA7000F014FDC8211A
:10895000304800F0A5FB282000F0BEFB0A2000F004
:10896000CEFB08E0D8208DF800006A4601214FF4C4
:108970000B6002F0CBF904F0020018B1D9208DF899
:10898000000002E0D8208DF800006A46012140F284
:108990003D7002F0BBF904F0040018B1012000F0B2
:1089A00069F802E0002000F065F804F0100018B14A
:1089B0000120FFF707FF02E00020FFF703FF44F06C
:1089C00008001549488101F08DFD00201249887387
:1089D00004F0400018B10846807B801D887304F4C1
:1089E000C07020B10C48807B801D0B49887304F057
:1089F000140020B10848807B10300749887304F0C8
:108A0000030020B10448807B001D034988730020C7
:108A10003EBD000009E3CA02640000243EB50446DE
:108A20006CB10EA1D1E900208968CDE90020029146
:108A30006A4609214FF4976002F068F93EBD0AA228
:108A4000D2E900109268CDE9010200916A4609213D
:108A50004FF4976002F05AF9F0E70000B8AAB38D1E
:108A6000B4980D355D000000B8AAAAAAB088C3C5A5
:108A7000C700000038B5044664B1C0208DF800007E
:108A8000C2208DF80100C4208DF80200C6208DF8A8
:108A9000030004E08B2204216846F7F77DFC6A4658
:108AA000042140F6982002F031F901F01BFD38BD99
:108AB00010B5C8234FF48062024940F6F63001F049
:108AC000A5FB10BDE8B000082DE9F04F8DB00746BA
:108AD000884615469946DDE9166B00240020308053
:108AE0006B49887B5A4605A901F05CFC18B1601EF1
:108AF0000DB0BDE8F08F6648807A00F014000028C1
:108B000067D09DF8140000069DF8151040EA01405A
:108B10009DF8161040EA01209DF8171008432860C0
:108B20009DF8180000069DF8191040EA01409DF8D4
:108B30001A1040EA01209DF81B10084368609DF858
:108B40001C0000069DF81D1040EA01409DF81E1013
:108B500040EA01209DF81F100843A8609DF82000FE
:108B600000069DF8211040EA01409DF8221040EADD
:108B700001209DF823100843E86004F11000C4B2FE
:108B8000286800140190686800140290A868001416
:108B90000390E8680014049001984043029901FB97
:108BA0000100039901FB0100049901FB010ABAF1DC
:108BB000706F02DBBAF1885F05DD01F093FC0020E5
:108BC0003080401E94E7B6F9000040F48070308099
:108BD00000BF2F48807A00F0400020B305A9601C38
:108BE000085C095D40EA012000B2A8F8000005A970
:108BF000E01C095C05AAA01C105C41EA002000B240
:108C0000A8F8020005A9601D095C201D105C41EA5E
:108C1000002000B2A8F80400A01DC4B2B6F90000FC
:108C200040F0080030801A48408900F4C07008B352
:108C300005A9601C085C095D40EA012000B238808B
:108C400005A9E01C095C05AAA01C105C41EA0020F3
:108C500000B2788005A9601D095C201D105C41EA06
:108C6000002000B2B880A01DC4B2B6F9000040F0E8
:108C7000700030800648807A00F0030018B105A922
:108C80000819FFF76DFD484600F040FE00202FE771
:108C90006400002470B588B0064601A801F000F910
:108CA000BDF804000021C90341EA5045C40300BFD8
:108CB0004448007A00F0030056F82000059041482F
:108CC000007A00F0040010B10598404205903D483C
:108CD000007AC0F3C10056F8200006903948007AA7
:108CE00000F0200010B10698404206903548007A06
:108CF000C0F3811056F8200007903248008900F434
:108D0000807010B10798404207900598C117A0FBEA
:108D1000042301FB043100FB0510810041EA92703D
:108D200005900698C117A0FB042301FB043100FB4A
:108D30000510810041EA927006900798C117A0FBC8
:108D4000042301FB043100FB0510810041EA92700D
:108D500007900598000E8DF808000598000C8DF816
:108D600009000598000A8DF80A000598C0B28DF830
:108D70000B000698000E8DF80C000698000C8DF87C
:108D80000D000698000A8DF80E000698C0B28DF806
:108D90000F000798000E8DF810000798000C8DF852
:108DA00011000798000A8DF812000798C0B28DF8DC
:108DB000130002AA0C214FF4257001F0A7FF08B0A0
:108DC00070BD00006400002430B585B0044616A2D2
:108DD00007CA02AB07C3C82C03DD4FF0FF3005B054
:108DE00030BDC82090FBF4F0401E85B2280A8DF8F3
:108DF0000000E8B28DF801006A46022140F2162018
:108E000001F084FF10B14FF0FF30E8E702AA0C2117
:108E100040F6C12001F07AFF10B14FF0FF30DEE7DD
:108E2000044884810020DAE7FEF2ABC4AAF1DFDF58
:108E3000BBAFDFDF640000241FB504464848007A5A
:108E400000F0030054F8200001904548007A00F03B
:108E5000040010B10198404201904148007AC0F3EB
:108E6000C10054F8200002903D48007A00F0200034
:108E700010B10298404202903948007AC0F3811044
:108E800054F8200003903648008900F4807010B137
:108E90000398404203903349019880FB0101800F01
:108EA00040EA810001902F49029880FB0110820066
:108EB00042EA917002902B49039880FB01108200D6
:108EC00042EA917003900198000E8DF8000001981D
:108ED000000C8DF801000198000A8DF8020001983D
:108EE000C0B28DF803006A4604214FF4747001F09B
:108EF0000DFF18B14FF0FF3004B010BD0298000E06
:108F00008DF800000298000C8DF801000298000A0C
:108F10008DF802000298C0B28DF803006A46042161
:108F20004FF4757001F0F2FE10B14FF0FF30E3E73F
:108F30000398000E8DF800000398000C8DF80100D6
:108F40000398000A8DF802000398C0B28DF8030060
:108F50006A4604214FF4767001F0D8FECCE7000099
:108F60006400002409E3CA0210B586B0044647A095
:108F70000068039046A00068029046A00068019037
:108F800045A00068009004F0030003A9085C8DF878
:108F9000140003A8C4F3C101405C8DF8150003A8B8
:108FA000C4F38111405C8DF8160004F0030002A99F
:108FB000085C8DF8100002A8C4F3C101405C8DF874
:108FC000110002A8C4F38111405C8DF8120005AABB
:108FD000032140F2264001F099FE18B14FF0FF3016
:108FE00006B010BD04AA032140F22A4001F08EFE13
:108FF00010B14FF0FF30F3E701980590009804900E
:1090000004F0040058B19DF8140040F001008DF800
:1090100014009DF8100040F001008DF8100004F0DD
:10902000200058B19DF8150040F001008DF81500A2
:109030009DF8110040F001008DF8110004F48070DB
:1090400058B19DF8160040F001008DF816009DF80B
:10905000120040F001008DF8120005AA03214FF420
:10906000886001F053FE10B14FF0FF30B8E704AA5A
:10907000032140F2314001F049FE10B14FF0FF30C2
:10908000AEE7064804810020AAE700004CCD6C0042
:109090000CC92C0036567600264666006400002473
:1090A000F8B505460E464FF47A7095FBF0F000FBDC
:1090B00006F4200E8DF80000200C8DF80100200A27
:1090C0008DF80200E0B28DF803006A4604214FF4E7
:1090D000AE7001F01BFEF8BD38B50446052094FBC8
:1090E000F0F084B220128DF80000E0B28DF801009B
:1090F0006A4602214FF4AD7001F008FE38BD38B564
:109100000446052094FBF0F084B220128DF8000094
:10911000E0B28DF801006A4602214FF4AC7001F014
:10912000F5FD38BD38B504460020009004F001007C
:1091300020B19DF8000040F03000009004F00200E3
:1091400020B19DF8000040F00C00009004F00400F5
:1091500020B19DF8000040F0030000906A46012114
:109160004FF4A47001F0D2FD38BD38B50446012C8F
:1091700001DA012402E0042C00DD0424601EC0B2E8
:1091800000906A46012140F24F1001F0BFFD38BD4A
:10919000F0B52DED028B83B006460F4606F00700B2
:1091A00010B1B7F5C86F05DD4FF0FF3003B0BDEC6F
:1091B000028BF0BD00EE107AB8EE400ADFED5B0ADC
:1091C00080EE208A01A800F045FE9DF804000228E8
:1091D00006D0042817D0082828D010284CD138E011
:1091E0009FED530A28EE000ABCEEC00A10EE100AEA
:1091F00084B29FED500A28EE000ABCEEC00A10EEC1
:10920000100A85B23BE09FED4C0A28EE000ABCEE46
:10921000C00A10EE100A84B29FED480A28EE000A38
:10922000BCEEC00A10EE100A85B228E09FED440A99
:1092300028EE000ABCEEC00A10EE100A84B29FEDC0
:10924000410A28EE000ABCEEC00A10EE100A85B2F0
:1092500015E09FED3D0A28EE000ABCEEC00A10EEB4
:10926000100A84B29FED390A28EE000ABCEEC00A4B
:1092700010EE100A85B202E04FF0FF3096E700BF13
:1092800020128DF80800E0B28DF8090028128DF840
:109290000A00E8B28DF80B0006F00100A0B102AAA6
:1092A00002214FF4EA7001F031FD10B14FF0FF30B0
:1092B0007CE70DF10A0202214FF4927001F026FDC5
:1092C00010B14FF0FF3071E706F00200A0B102AA22
:1092D00002214FF4EC7001F019FD10B14FF0FF3096
:1092E00064E70DF10A0202214FF4947001F00EFDC3
:1092F00010B14FF0FF3059E706F00400A0B102AA08
:1093000002214FF4EE7001F001FD10B14FF0FF307B
:109310004CE70DF10A0202214FF4967001F0F6FCC1
:1093200010B14FF0FF3041E700203FE70000484315
:109330000000804600004046000000460000C04596
:109340000000804500004045000000450000C0448A
:1093500038B50446052094FBF0F085B228128DF84C
:109360000000E8B28DF801006A4602214FF4EF7068
:1093700001F0CCFC38BD38B50446052094FBF0F074
:1093800085B228128DF80000E8B28DF801006A4617
:1093900002214FF4ED7001F0B9FC38BD82B0CDE987
:1093A000000121F0004001909DED000B02B051EC56
:1093B000100B704713B50C464FF6FF730122694638
:1093C0000248FCF733F900981CBD00001403002488
:1093D0007CB505462E494968087801AB04220D2169
:1093E000FCF756FB08B107207CBD9DF80700C0F3D1
:1093F00001109DF8041001F0E00140EAE1008DF851
:1094000000009DF80700C0F381009DF8051001F0F1
:10941000E00140EAE1008DF801009DF8070000F04E
:1094200003009DF8061001F0E00140EAE1008DF82C
:109430000200002427E01DF8040030B99FED150A52
:1094400005EB840080ED000A1BE09FED130A05EB9D
:10945000840080ED000A0BE005EB840090ED000A2B
:10946000DFED0E0A20EE200A05EB840080ED000AF5
:109470001DF80400401EC0B20DF804000028EBD116
:1094800000BF601CC4B2032CD5DB0020ACE7000099
:1094900000000024000000007B14AE3E1D5A843FF3
:1094A0002DE9F04F87B005460C46914601208DF816
:1094B000100000208DF81100FE4A1268517DFD4A0F
:1094C0005268107804AB0222FCF786FB20B14FF003
:1094D000FF3007B0BDE8F08FC820F8F7F5F800209E
:1094E0008DF81000F34A1268517CF24A52681078E5
:1094F00004AB0122FCF770FB10B14FF0FF30E8E73E
:10950000EC4A12685179EB4A5268107804AB012298
:10951000FCF762FB10B14FF0FF30DAE7E54A126862
:10952000517DE44A5268107804AB0122FCF754FBE9
:1095300010B14FF0FF30CCE7DE4A1268917EDD4A71
:109540005268107804AB0122FCF746FB10B14FF0D3
:10955000FF30BEE7D74A12681179D64A52681078B0
:1095600004AB0122FCF738FB10B14FF0FF30B0E73D
:109570000C208DF81000CF4A12681179CD4A52683C
:10958000107804AB0122FCF727FB10B14FF0FF303D
:109590009FE70F20F8F798F8C648806A407A8DF860
:1095A0001000C44A12689178C24A5268107804AB1D
:1095B0000122FCF711FB10B14FF0FF3089E7BD48E5
:1095C000806A007A8DF81000BA4A12685178B94A58
:1095D0005268107804AB0122FCF7FEFA10B14FF08C
:1095E000FF3076E7B9F1000F07D0B248806A807A81
:1095F00040F0E0008DF8100004E0AE48806A807A08
:109600008DF81000AB4A12689179AA4A5268107816
:1096100004AB0122FCF7E0FA10B14FF0FF3058E73D
:10962000B9F1000F07D0A348806AC07A40F0E0008B
:109630008DF8100003E0A048C07A8DF810009D4A14
:109640001268D1799B4A5268107804AB0122FCF76A
:10965000C3FA10B14FF0FF303BE7B9F1000F02D071
:10966000C820F8F731F840208DF81000914A1268B0
:109670001179904A5268107804AB0122FCF7ACFAD9
:1096800010B14FF0FF3024E778208DF81000894AA0
:1096900012685179874A5268107804AB0122FCF7AE
:1096A0009BFA10B14FF0FF3013E783498889F8F730
:1096B0000BF800208DF810007E4A126851797D4A1F
:1096C0005268107804AB0122FCF786FA10B14FF013
:1096D000FF30FEE6774A1268117B764A52681078AE
:1096E00004AB0222FCF7D4F910B14FF0FF30F0E6E2
:1096F0009DF811009DF8101040EA012B0C209BFBF7
:10970000F0F0C6B20020A86068602860A0606060C9
:109710002060824665E0674A1268517B654A52685C
:10972000107804AB0C22FCF7B3F910B14FF0FF3006
:10973000CFE69DF811009DF8101040EA012000B21C
:10974000ADF808009DF813009DF8121040EA0120C2
:1097500000B2ADF80A009DF815009DF8141040EA1B
:10976000012000B2ADF80C00BDF9081020680844D3
:109770002060BDF90A10606808446060BDF90C10F3
:10978000A0680844A0609DF817009DF8161040EAF4
:10979000012000B2ADF800009DF819009DF81810E6
:1097A00040EA012000B2ADF802009DF81B009DF8D0
:1097B0001A1040EA012000B2ADF80400BDF9001013
:1097C000286808442860BDF9021068680844686089
:1097D000BDF90410A8680844A8600AF1010000F06F
:1097E000FF0AB24597DB3448D0F800C02868C1179B
:1097F000090441EA10410704624600233846F6F79F
:109800009AFD32460023CDE90201F6F794FD286067
:109810002948D0F800C06868C117090441EA10411E
:109820000704624600233846F6F785FD32460023DA
:10983000CDE90201F6F77FFD68601F48D0F800C04F
:10984000A868C117090441EA1041070462460023D1
:109850003846F6F770FD32460023CDE90201F6F7EF
:109860006AFDA8601448D0F804C02068C117090434
:1098700041EA10410704624600233846F6F75BFDD3
:1098800032460023CDE90201F6F755FD20600A4873
:10989000D0F804C06068C117090441EA1041070408
:1098A000624600233846F6F746FD32460023CDE9EE
:1098B000020103E000000024C0B00008F6F73BFD01
:1098C00060601148D0F804C0A068C117090441EADB
:1098D00010410704624600233846F6F72CFD324655
:1098E0000023CDE90201F6F726FDA060A06800285C
:1098F00004DDA068A0F58030A06003E0A06800F55A
:109900008030A0600020E4E5C0B0000810B5044637
:10991000F7F7F8FF2060002010BD0000012001498A
:10992000C870704774000024F0B52DED048B81B031
:1099300006460F4600253F49496808786B460322D2
:109940000D21FCF7A5F820B1072001B0BDEC048B78
:10995000F0BD9DF8000000F01F008DF800009DF89C
:10996000010000F01F008DF801009DF8020000F0DA
:109970001F008DF80200002457E056F8241057F815
:109980002420881A002801DB014600E0414200EE55
:10999000101AB8EEC00ADFED280A80EE208A1DF802
:1099A000040070B3254890ED000AB8EE400ADFEDE0
:1099B000240A80EE801AB0EE419A05E09FED210A5C
:1099C00029EE000AB0EE409A1DF80400401EC0B215
:1099D0000DF804000028F1D188EE090AF7EE000A1C
:1099E00070EE608A00BFB0EEE80A1448D0ED060AB7
:1099F000B4EEE00AF1EE10FA16DD0120A0400543B6
:109A000012E0FFE70D4890ED040AB4EEC80AF1EE4B
:109A100010FA06DC90ED050AB4EEC80AF1EE10FA71
:109A200002D20120A0400543641C032CA5DB28467C
:109A30008BE700000000002400008047C0B0000851
:109A400000B04C4554E3853F014691F90020002ABF
:109A500001DD00201EE091F90020002A01DA042037
:109A600018E091F90120002A01DD012012E091F9AE
:109A70000120002A01DA05200CE091F90220002AD9
:109A800001DD022006E091F90220002A01DA062019
:109A900000E0072070470000B8B0F8F797FAFCF72D
:109AA00099FEFCF7BDF9FCF76BF9FCF739FAFCF706
:109AB000C1FAFCF7DBFAFCF751FBFCF795FBFCF76E
:109AC000D9FBFCF75BFAFCF787FA6920AE4908601E
:109AD000D320AE490860D220AD4908600120AD49CD
:109AE0000860F6F79BFF6820A7490860D120A749C6
:109AF0000860D020A64908600120A6490860F6F752
:109B00008DFF6820A0490860D120A0490860D020BE
:109B10009F49086002209F490860F6F77FFF69208F
:109B200099490860D32099490860D2209849086073
:109B3000022098490860F6F771FF69209249086091
:109B4000D32092490860D2209149086003209149AE
:109B50000860F6F763FF68208B490860D1208B49C5
:109B60000860D0208A49086003208A490860F6F717
:109B700055FF8948F8F71AFB012404E1012C7DD137
:109B8000692081490860D32080490860D22080493B
:109B9000086001207F49086035AA36A937A8FCF77C
:109BA0002FFD054623AA24A925A8FCF7BDF87BA014
:109BB000DDE923322599FDF789FD9DED260AB7EEF3
:109BC000C00A8DED200B9DED270AB7EEC00A8DED82
:109BD0001E0B9DED280AB7EEC00A8DED1C0B9DED06
:109BE000290AB7EEC00A8DED1A0B9DED2A0AB7EED1
:109BF000C00A8DED180B9DED2B0AB7EEC00A8DED56
:109C0000160B9DED2C0AB7EEC00A8DED140B9DEDE1
:109C10002D0AB7EEC00A8DED120B9DED2E0AB7EEA0
:109C2000C00A8DED100B9DED2F0AB7EEC00A8DED29
:109C30000E0B9DED300AB7EEC00A8DED0C0B9DEDBD
:109C4000310AB7EEC00A8DED0A0B9DED320AB7EE70
:109C5000C00A8DED080B9DED330AB7EEC00A8DEDFD
:109C6000060B9DED340AB7EEC00A8DED040B9DED99
:109C7000350AB7EEC00A8DED020B00E010E09DED55
:109C8000360AB7EEC00A8DED000B9DED370AB7EE30
:109C9000C00A53EC102B44A0FDF718FD02246DE020
:109CA000022C13D1682038490860D1203749086058
:109CB000D0203749086001203649086032AA33A90C
:109CC00034A8FCF79DFC0546032457E0032C13D170
:109CD00068202D490860D1202C490860D0202C49EB
:109CE000086002202B4908602FAA30A931A8FCF790
:109CF00087FC0546042441E0042C13D16920224945
:109D00000860D32021490860D22021490860022040
:109D1000204908602CAA2DA92EA8FCF771FC054645
:109D200005242BE0052C13D1682017490860D120A9
:109D300016490860D02016490860032015490860BC
:109D400029AA2AA92BA8FCF75BFC0546062415E0E6
:109D5000062C13D169200C490860D3200B490860F8
:109D6000D2200B49086003200A49086026AA27A9C7
:109D700028A8FCF745FC0546012400BF0122510339
:109D80001748F7F7B3FDF9E6380000243C0000243B
:109D90004000002444000024E401002425642C2514
:109DA000642C25640000000025662C25662C2566A1
:109DB0002C25662C25662C25662C25662C25662CE4
:109DC00025662C25662C25662C25662C25662C25DB
:109DD000662C25662C25662C25662C25660D0A002A
:109DE0000008025870B50446002624F00104184803
:109DF00090F8240008B1002070BD1548807A10B991
:109E00004FF0FF30F8E71248057C807A2040104977
:109E100008740846007CA04202D04FF0FF3600E0F4
:109E2000002614B90A48007D18B1012001F0B4F8E9
:109E300002E0002001F0B0F83CB100F053FB20B18B
:109E4000034805744FF0FF30D6E73046D4E70000F2
:109E50000000002401461148407A30B1012807D0A3
:109E6000022808D003280CD108E0022008700BE07B
:109E70000420087008E00820087005E01020087031
:109E800002E04FF0FF30704700BF0448C07C18B1BB
:109E900008784006000E08700020F4E70000002457
:109EA00001461348407A30B1012808D002280AD070
:109EB000032810D10BE04FF4804008800EE041F6FB
:109EC0009C7008800AE04FF48050088006E04FF450
:109ED0000060088002E04FF0FF30704700BF044888
:109EE000C07C10B10888401008800020F5E7000011
:109EF0000000002401460248007C087000207047E2
:109F00000000002401460F48007A30B1012807D034
:109F1000022809D003280FD10AE0FA2008800EE0B9
:109F20004FF4FA7008800AE04FF47A70088006E077
:109F30004FF4FA60088002E00020088000BF00BFF4
:109F4000002070470000002401461248007A30B11A
:109F5000012809D002280CD0032814D10EE09FED6F
:109F60000E0A81ED000A11E09FED0C0A81ED000A56
:109F70000CE09FED0B0A81ED000A07E09FED090A56
:109F800081ED000A02E04FF0FF30704700BF002073
:109F9000FBE70000000000240000034300008342B0
:109FA000333303423333834101461248C07A0828D1
:109FB00017D2DFE800F01704070A0D101318BC20B1
:109FC000088013E06220088010E02A2008800DE05D
:109FD000142008800AE00A20088007E00520088095
:109FE00004E000BF00BF0020088000BF00BF0020C9
:109FF00070470000000000240146064890F8240045
:10A0000010B14FF0FF3070470248C089088000202F
:10A01000F9E70000000000247CB5054680208DF89B
:10A020000000664A1268517D644A526810786B4697
:10A030000122FBF7D1FD10B14FF0FF307CBD642051
:10A04000F7F742FB00208DF800005C4A1268517D52
:10A050005A4A526810786B460122FBF7BDFD10B1D9
:10A060004FF0FF30EAE7554A1268517E534A526872
:10A0700010786B460622FBF70BFD10B14FF0FF3056
:10A08000DCE79DF80500C007400F9DF8031001F0C4
:10A09000010140EA41009DF8011001F0010140EA90
:10A0A000010494B1012C03D101214448C17431E071
:10A0B000022C03D100214148C1742BE0214640A06D
:10A0C000FDF704FB4FF0FF30B8E73C4A1268D17847
:10A0D0003A4A526810786B460122FBF7D9FC10B15E
:10A0E0004FF0FF30AAE79DF8000000F00F042CB9F4
:10A0F0003D48FDF7EBFA4FF0FF309FE7042C06D107
:10A100003AA0FDF7E3FA01212C48C17402E00021D6
:10A110002A48C174FF2129488172FF20274908720B
:10A12000FF2126484172C1724FF6FF71C181FF21A4
:10A13000017481740121017380F82210002180F8DC
:10A140002310417501751630016041608160163839
:10A1500080F8241080F82510C1844FF4FA6000F0D4
:10A1600063FC10B14FF0FF3068E7022000F02CFBD9
:10A1700010B14FF0FF3061E72A2000F0CFFC10B1A2
:10A180004FF0FF305AE7322000F00AFD10B14FF0D7
:10A19000FF3053E70020FFF725FE10B14FF0FF30EE
:10A1A0004CE7002000F052FB10B14FF0FF3045E7C4
:10A1B000002000F043FD002040E7000000000024E4
:10A1C000556E737570706F7274656420736F66740A
:10A1D000776172652070726F647563742072657642
:10A1E0002025642E0A00000008BE000848616C6645
:10A1F0002073656E73697469766974792070617211
:10A200007420666F756E642E0A0000002DE9F0431D
:10A2100085B005460E4690469946294890F8250097
:10A2200020B14FF0FF3005B0BDE8F08316B94FF014
:10A23000FF30F8E7002423E0281B102801DD102060
:10A2400000E0281B87B232193946204600F05EFD37
:10A2500010B14FF0FF30E6E701AA3946204600F082
:10A2600001F910B14FF0FF30DDE730193A4601A98E
:10A27000F6F7A4F810B16FF00100D4E7E01984B24A
:10A28000AC42D9DB4FEA28208DF8000008F0FF002F
:10A290008DF801000A4A1268517F094A5268107805
:10A2A0006B460222FBF798FC10B14FF0FF30BAE783
:10A2B0000121034880F82510A0F826900020B2E77D
:10A2C0000000002438B50446282C02DD4FF0FF3092
:10A2D00038BDDCB9002000F0EBFB00208DF8000059
:10A2E00007208DF801002E4A1268517D2C4A5268D1
:10A2F00010786B460222FBF76FFC10B14FF0FF3075
:10A30000E6E70021264801750020E1E7012000F082
:10A31000CFFB20208DF80000012C06D100208DF805
:10A320000100052000F0FAFB17E0052C06DC0120F7
:10A330008DF80100052000F0F1FB0EE0142C06DC86
:10A3400002208DF801000A2000F0E8FB05E0032060
:10A350008DF80100142000F0E1FB9DF801000721B9
:10A3600001EB8010C0B28DF801000D4A1268517DDA
:10A370000B4A526810786B460222FBF72DFC10B195
:10A380004FF0FF30A4E708210548817200210173D6
:10A39000012101750020FFF725FD002098E700004E
:10A3A00000000024F8B504460F4616462C4890F8E5
:10A3B000240010B94FF0FF30F8BD2948807A10B959
:10A3C0004FF0FF30F8E7264A1268117B244A5268A2
:10A3D00010786B460222FBF75BFB10B14FF0FF30A9
:10A3E000EAE79DF801009DF8001040EA0125A5422A
:10A3F00003DA00203070401EDEE7194840684088CC
:10A40000B5EB600F17DD164A1268D17C144A52680A
:10A4100010786B460122FBF73BFB10B14FF0FF3089
:10A42000CAE79DF8000000F0100020B100F05AF8D3
:10A430006FF00100C0E7E2B2094B1B68597B084B83
:10A440005B6818783B46FBF723FB10B14FF0FF30F9
:10A45000B2E795FBF4F0401E30700020ACE700003E
:10A4600000000024F8B504460D46164616B94FF014
:10A47000FF30F8BD1A48807A10B94FF0FF30F8E786
:10A4800020128DF80000E0B28DF801009DF8010067
:10A490002844134949684989884202DD4FF0FF305A
:10A4A000E7E70F4A1268D17E0D4A526810786B4672
:10A4B0000222FBF791FB10B14FF0FF30D9E7EAB26F
:10A4C000074B1B68197E064B5B6818783346FBF711
:10A4D000DFFA10B14FF0FF30CBE70020C9E70000F2
:10A4E0000000002408B57048807A10B94FF0FF30A2
:10A4F00008BD002000906C4A1268517C6A4A52687C
:10A5000010786B460122FBF767FB10B14FF0FF306C
:10A51000EEE7654A12685179634A526810786B46D3
:10A520000122FBF759FB10B14FF0FF30E0E75E4A24
:10A53000126811795C4A526810786B460122FBF769
:10A540004BFB10B14FF0FF30D2E7574890F8240092
:10A55000002853D00C200090534A12681179524AB7
:10A56000526810786B460122FBF736FB10B14FF0B2
:10A57000FF30BDE73220F7F7A7F8C02000904A4827
:10A58000807A00F0010020B19DF8000040F020002A
:10A590000090454A12681179434A526810786B4618
:10A5A0000122FBF719FB10B14FF0FF30A0E73E4846
:10A5B000407C10B10220009001E0002000903A4A57
:10A5C0001268517C384A526810786B460122FBF7BA
:10A5D00003FB10B14FF0FF308AE700200090324AB1
:10A5E00012685179304A526810786B460122FBF7A5
:10A5F000F3FA002855D04FF0FF3079E7042000909F
:10A60000294A12681179284A526810786B4601224B
:10A61000FBF7E2FA10B14FF0FF3069E72248807C87
:10A6200020B92148807A00F0010010B94020009044
:10A6300001E0602000901C4A126811791A4A5268A1
:10A6400010786B460122FBF7C7FA10B14FF0FF30CC
:10A650004EE73220F7F738F81348407C10B101205C
:10A66000009001E0002000900F4A1268517C0E4AD1
:10A67000526810786B460122FBF7AEFA10B14FF02A
:10A68000FF3035E7084A12685179074A5268107856
:10A69000054B10330122FBF79FFA10B14FF0FF304A
:10A6A00026E7002024E70000000000242DE9F04FF9
:10A6B0008DB083460F4602200C90424890F824004B
:10A6C00020B1002000F068F9012600E0002603A870
:10A6D000FFF718FC05A8FFF7BDFB01A8FFF764FC16
:10A6E00002A8FFF789FC374890F80AA004A8FFF7F2
:10A6F00001FC002407E0002239465846FEF7D0FE50
:10A7000000B902E0641C022CF5DB00BF022C01D171
:10A71000002528E0002407E0012206A909A8FEF789
:10A72000BFFE00B902E0641C022CF5DB00BF022C66
:10A7300001D1002517E006A93846FDF7A9FF00F072
:10A74000FF0809A95846FFF7EFF800F0FF090025B8
:10A75000B9F1000F01D145F00105B8F1000F01D1A9
:10A7600045F0020500BFFF2016490872FF21154879
:10A770004172C1724FF6FF71C181FF218172017474
:10A7800001210173BDF80C0000F04EF99DF8140092
:10A7900000F01AF8BDF8040000F0C0F9BDF8080098
:10A7A00000F0FEF9504600F049FA9DF81000FFF75E
:10A7B00019FB16B1012000F0EFF828460DB0BDE8F6
:10A7C000F08F00000000002438B504461E48807A4F
:10A7D00010B94FF0FF3038BD022C06D0042C07D042
:10A7E000082C08D0102C0CD108E0002000900BE0C1
:10A7F0000820009008E01020009005E0182000904C
:10A8000002E04FF0FF30E6E700BF0F48407A9DF8C6
:10A810000010B0EBE10F01D10020DCE70A4A12681A
:10A82000D179094A526810786B460122FBF7D4F9B6
:10A8300010B14FF0FF30CEE79DF80000C110024884
:10A8400041720020C7E700000000002438B504462C
:10A850005048807CA04201D1002038BD002C46D059
:10A860004C4A126811794B4A526810786B460122A3
:10A87000FBF70EF910B14FF0FF30EEE79DF8000046
:10A8800020F020000090434A12681179414A526832
:10A8900010786B460122FBF79FF910B14FF0FF30A3
:10A8A000DBE70320F6F710FF02200090394890F80C
:10A8B000220020B19DF8000040F080000090354853
:10A8C00090F8230020B19DF8000040F03000009087
:10A8D000304A1268D17D2F4A526810786B460122A7
:10A8E000FBF77AF9002851D04FF0FF30B5E7294A3D
:10A8F00012681179274A526810786B460122FBF7DB
:10A90000C7F810B14FF0FF30A7E72248807A00F077
:10A91000010028B19DF8000040F02000009004E004
:10A920009DF8000020F0200000901A4A126811796A
:10A93000184A526810786B460122FBF74DF910B1A6
:10A940004FF0FF3089E70320F6F7BEFE114890F87C
:10A95000220010B18020009001E0002000900D48FE
:10A9600090F8230020B19DF8000040F030000090E6
:10A97000084A1268D17D074A526810786B46012256
:10A98000FBF72AF910B14FF0FF3066E701488474F5
:10A99000002062E70000002438B50446214890F802
:10A9A0002400A04201D1002038BD24B31D4890F8F6
:10A9B000250010B94FF0FF30F6E7002000F0ECFA68
:10A9C0000020FFF743FF1749C88C00F0E9F800208A
:10A9D00000901449496808786B4601222321FBF74F
:10A9E000FBF801210F4880F82410012000F0D4FA70
:10A9F000FFF778FD13E0002000F0CEFA0948007C54
:10AA000000900849496808786B4601222321FBF72A
:10AA1000E3F80021034880F82410FFF763FD0020CD
:10AA2000C2E700000000002438B504461F48807AC1
:10AA300010B94FF0FF3038BDFA2C09D0B4F5FA7FC9
:10AA400009D0B4F57A7F09D0B4F5FA6F0CD108E0DB
:10AA5000002000900BE00820009008E010200090FB
:10AA600005E01820009002E04FF0FF30E3E700BF60
:10AA70000E48007A9DF80010B0EBE10F01D10020E4
:10AA8000D9E70A4A12689179084A526810786B46E9
:10AA90000122FBF7A1F810B14FF0FF30CBE79DF892
:10AAA0000000C010014908720020C4E70000002423
:10AAB00038B50446184890F82300A04201D1002080
:10AAC00038BD14B13020009001E000200090124801
:10AAD000807C20B19DF8000040F0020000900E48FC
:10AAE00090F8220020B19DF8000040F08000009016
:10AAF000094A1268D17D084A526810786B460122D3
:10AB0000FBF76AF810B14FF0FF30D9E7024880F840
:10AB100023400020D4E700000000002438B504469C
:10AB20001E48807A10B94FF0FF3038BDBC2C02DBD4
:10AB30000120009015E0622C02DB0220009010E062
:10AB40002A2C02DB032000900BE0142C02DB0420F3
:10AB5000009006E00A2C02DB0520009001E00620B0
:10AB600000900E48C07A9DF80010884201D1002064
:10AB7000DBE70A4A12689178084A526810786B46F7
:10AB80000122FBF729F810B14FF0FF30CDE79DF817
:10AB900000100248C1720020C7E700000000002436
:10ABA00038B504462448807A10B94FF0FF3038BDDC
:10ABB000214890F8240010B14FF0FF30F7E71E480D
:10ABC000007D50B134B1282C04DCE0B2FFF77AFBF1
:10ABD0000020ECE70020FFF775FB042C01DA0424C9
:10ABE00004E0B4F57A7F01DD4FF47A744FF47A70A3
:10ABF00090FBF4F0401EC0B200900F4A12685178EA
:10AC00000D4A526810786B460122FAF7E5FF10B141
:10AC10004FF0FF30CBE79DF80000401C4FF47A71F5
:10AC200091FBF0F081B20448C1810146C989481006
:10AC3000FFF774FF0020BAE70000002438B504468F
:10AC400004F0700010B10120009005E014B1002064
:10AC5000009001E0402000902B4A1268517D2A4A62
:10AC6000526810786B460122FAF7B6FF20B1002136
:10AC700025488172481E38BD9DF8000020F0400133
:10AC8000214801730020009004F0400020B99DF895
:10AC9000000040F00400009004F0200020B99DF86E
:10ACA000000040F00200009004F0100020B99DF870
:10ACB000000040F00100009004F0080020B99DF869
:10ACC000000040F0380000900F4A1268917D0E4A53
:10ACD000526810786B460122FAF77EFF20B10021FE
:10ACE00009488172481EC6E724B1082C02D0002012
:10ACF000FFF7DEFE04488472002101753220F6F76A
:10AD0000E3FC0020B7E7000000000024F8B504468B
:10AD10000D46164616B94FF0FF30F8BD1A48807A36
:10AD200010B94FF0FF30F8E720128DF80000E0B2C4
:10AD30008DF801009DF801002844134949684989AC
:10AD4000884202DD4FF0FF30E7E70F4A1268D17EFC
:10AD50000D4A526810786B460222FAF73DFF10B197
:10AD60004FF0FF30D9E7EAB2074B1B68197E064B5C
:10AD70005B6818783346FAF72FFF10B14FF0FF30B9
:10AD8000CBE70020C9E700000000002410B58AB01E
:10AD90000020099003A906A8FFF788FC0446072CA9
:10ADA0003FD102A8FFF7D0F89DED060AB8EEC00A21
:10ADB000DDED020A20EE200ABDEEC00A8DED060A86
:10ADC0009DED070AB8EEC00ADDED020A20EE200A6A
:10ADD000BDEEC00A8DED070A9DED080AB8EEC00A67
:10ADE000DDED020A20EE200ABDEEC00A8DED080A54
:10ADF00006A8FEF721F801A8FFF752F8BDF80410E5
:10AE0000039848430390BDF8041004984843049005
:10AE1000BDF8041005984843059003A8FDF73AFFD4
:10AE200000BF74208DF82400E0B28DF8250009A938
:10AE3000062000F002F80AB010BD70B586B00546D5
:10AE40000C46142101A8F5F7AEFA24208DF8040071
:10AE50008DF805500DB1012D17D120460188090A42
:10AE60008DF8061001788DF807104188090A8DF8D1
:10AE7000081081788DF809108188090A8DF80A1068
:10AE800001798DF80B10082683E0022D3ED1204673
:10AE90000168090E8DF806100168090C8DF807107D
:10AEA0000188090A8DF8081001788DF809104168A9
:10AEB000090E8DF80A104168090C8DF80B10818875
:10AEC000090A8DF80C1001798DF80D108168090EB2
:10AED0008DF80E108168090C8DF80F100189090A90
:10AEE0008DF81010017A8DF81110C168090E8DF8D7
:10AEF0001210C168090C8DF813108189090A8DF8A8
:10AF00001410017B8DF81510122642E0032D07D195
:10AF100020788DF8060060788DF80700042638E068
:10AF2000042D04D120788DF80600032631E0052D8C
:10AF300020D120460168090E8DF806100168090C21
:10AF40008DF807100188090A8DF8081001788DF82E
:10AF500009104168090E8DF80A104168090C8DF836
:10AF60000B108188090A8DF80C1001798DF80D10ED
:10AF70000A260EE0062D0CD120788DF806006078A8
:10AF80008DF80700A0788DF80800E0788DF80900AA
:10AF9000062606B070BD000038B50446214890F87A
:10AFA0002400C0B114B10220009001E00020009004
:10AFB0001C4A1268517C1B4A526810786B46012269
:10AFC000FAF70AFE10B14FF0FF3038BD9DF80010BF
:10AFD0001448417423E01348807A10B94FF0FF30D1
:10AFE000F3E724B10F48407C08B10020EDE714B12D
:10AFF0000120009001E0002000900A4A1268517C74
:10B00000084A526810786B460122FAF7E5FD10B144
:10B010004FF0FF30D9E79DF800100248417400203E
:10B02000D3E700000000002400B541EC100B2DED2B
:10B03000028B83B0B1EEC08B18EE100A18EE901A96
:10B040008DED008B002818BF0120084320F0004040
:10B05000C0F17F6000F1E040C00F14D010EE101A74
:10B0600010EE900A8DED000B002918BF0121084356
:10B0700020F00040C0F17F6000F1E040C00F04BF4D
:10B080000120FCF7B9FE51EC180B03B0BDEC028BAC
:10B0900000BD000075191A0C6A231B1C00001F203C
:10B0A0007274433B4138393A006B6C376F06246D3C
:10B0B0006E706800000476005401F7FD0001000086
:10B0C00083000000000800000001001832000500A5
:10B0D000000020410000D242295C0F3E9A99993E1F
:10B0E0003333733F295C0F3E0000700000000024E2
:10B0F000000000020003000000650054FFEF0000A4
:10B10000FA80000B12820001030C30C30E8C8CE914
:10B1100014D5400213710F8E3883F8833000F88302
:10B12000258EF8833000F883FFFFFFFF0FFEA9D6BE
:10B13000240004001A8279A10000003CFFFF0000F7
:10B140000010000038836FA2003E03304000000072
:10B1500002CAE3093E800000200000000000000059
:10B160004000000060000000000C0000000C186EA1
:10B17000000006920A16C0DFFFFF0256FD8CD3774F
:10B18000FFE1C496E0C5BEAA00000000FFFF0B2B44
:10B1900000001657000003594000000000001DFA8F
:10B1A00000026C1D000000003FFFDFEB003EB3B665
:10B1B000000D227800002F3C00000000001942B56D
:10B1C000000039A20000B365D90E9FC91DCF4C34D1
:10B1D00030000000500000003BB67AE80064000038
:10B1E00000C8000000000000100000001000FA92EB
:10B1F0001000225E000D229F0001000000320000BE
:10B20000FF46000063D400001000000004D60000D8
:10B2100004CC000004CC00000000107200000040CC
:10B22000000000000000000000060002000500070A
:10B2300000000000006400000000000000000005A5
:10B240000005006400200000000000000000000075
:10B25000000040000000030000000032F8980000E9
:10B26000FF650000830F0000FF9BFC000000000052
:10B2700000000000000000000000000000000000CE
:10B2800000000000000000000000000000000000BE
:10B290000000000000001000400000000000000658
:10B2A0000000B26A000200000001FB830068000099
:10B2B00000D9FC007CF1FF83000000000065000065
:10B2C000006403E80064002800000025000000007E
:10B2D00016A000000000100000001000002F000069
:10B2E000000001F40000100000280000FFFF45816D
:10B2F000FFFFFA720000000000000000004400059B
:10B300000005BAC6004778A2000000010000000056
:10B3100000000600000000140000254D002F706D95
:10B32000000005AE000C02D000000000000000008C
:10B330000000000000000000001B000000000000F2
:10B340000000000000000000006400000008000091
:10B3500000000000000000000000000000000000ED
:10B3600000000000000000000000000000000000DD
:10B3700000000000000000000000000000000000CD
:10B3800000000000000000000000000000000000BD
:10B3900000000000000000000000000000000000AD
:10B3A0000000000000000000001B00000000000082
:10B3B00000000000000E000E00000AC7000400009C
:10B3C00000000032FFFFFF9C00000B2B000000027A
:10B3D0000000000100000064FFE500000000000024
:10B3E000000000000000000000000001000000005C
:10B3F000000100000000000000018000000180004A
:10B4000000018000002426D300000000000000009E
:10B41000000600100096003C000000000000000044
:10B4200000000000000000000C0A4E68CDCF770934
:10B4300050166759C619CE820000000000000000B7
:10B4400000000000000000000000000000000000FC
:10B4500017D7840003000000000000000000000077
:10B46000C7938F9D1E1B1C190000000000000000E8
:10B4700000000000000000000000000000000000CC
:10B4800002031885000040000000000300000003D4
:10B49000000000000000000040000000000000006C
:10B4A000000000000000000000000000000000009C
:10B4B000000000000000000000000000000000008C
:10B4C000000000000000000000000000677DDF7E3B
:10B4D00072902E554CF6E688000000000000000037
:10B4E0000000000000000000D8DCB4B8B0D8B9AB50
:10B4F000F3F8FAB3B7BB8E9EAEF132F51BF1B4B8D8
:10B50000B08097F1A9DFDFDFAADFDFDFF2AAC5CDC8
:10B51000C7A90CC92C97F1A989264666B28999A9B1
:10B520002D557DB0B08AA896365676F1BAA3B4B23E
:10B5300080C0B8A89711B28398BAA3F02408441029
:10B540006418B2B9B49883F1A329557DBAB5B1A3F3
:10B550008393F0002850F5B2B6AA839328547CF167
:10B56000B9A3829361BAA2DADEDFDB819AB9AEF5C4
:10B57000606870F1DABAA2DFD9BAA2FAB9A38292EE
:10B58000DB31BAA2D9BAA2F8DF85A4D0C1BBAD83A2
:10B59000C2C5C7B8A2DFDFDFBAA0DFDFDFD8D8F1CE
:10B5A000B8AAB38DB4980D355DB2B6BAAF8C961902
:10B5B0008F9FA70E161EB49AB8AA872C547CBAA4E3
:10B5C000B08AB691325676B28494A4C808CDD8B861
:10B5D000B4B0F19982A82D557D98A80E161EA22C04
:10B5E000547C92A4F02C5078F184A898C4CDFCD857
:10B5F0000DDBA8FC2DF3D9BAA6F8DABAA6DED8BAC4
:10B60000B2B68696A6D0F3C841DAA6C8F8D8B0B4C8
:10B61000B882A892F52C548898F135D9F418D8F14D
:10B62000A2D0F8F9A884D9C7DFF8F883C5DADF69B2
:10B63000DF83C1D8F40114F1A8824EA884F311D19C
:10B6400082F5D992289788F109F41C1CD884A8F3B4
:10B65000C0F9D1D99782F129F40DD8F3F9F9D1D9EC
:10B6600082F4C203D8DEDF1AD8F1A2FAF9A88498CE
:10B67000D9C7DFF8F8F883C7DADF69DFF883C3D802
:10B68000F40114F198A8822EA884F311D182F5D97F
:10B6900092509788F109F41CD884A8F3C0F8F9D126
:10B6A000D99782F149F40DD8F3F9F9D1D982F4C4CC
:10B6B00003D8DEDFD8F1AD8898CCA809F9D98292F9
:10B6C000A8F57CF1883ACF944A6E98DB6931DAADFF
:10B6D000F2DEF9D88795A8F221D1DAA5F9F417D9C5
:10B6E000F1AE8ED0C0C3AE82C684C3A88595C8A56E
:10B6F00088F2C0F1F4010EF18E9EA8C63E56F554B4
:10B70000F18872F40115F19845856EF58E9E0488D6
:10B71000F142985A8E9E068869F4011CF1981E1118
:10B7200008D0F504F11E970202983625DBF9D98579
:10B73000A5F3C1DA85A5F3DFD88595A8F309DAA5C5
:10B74000FAD88292A8F578F1881A849F26889821E1
:10B75000DAF41DF3D8879F39D1AFD9DFDFFBF9F4D5
:10B760000CF3D8FAD0F8DAF9F9D0DFD9F9D8F40B1C
:10B77000D8F3879F39D1AFD9DFDFF41DF3D8FAFCB6
:10B78000A869F9F9AFD0DADEFAD9F88F9FA8F1CC21
:10B79000F398DB45D9AFDFD0F8D8F18F9FA8CAF373
:10B7A0008809DAAF8FCBF8D8F2AD978D0CD9A5DF29
:10B7B000F9BAA6F3FAF412F2D8950DD1D9BAA6F3D4
:10B7C000FADAA5F2C1BAA6F3DFD8F1BAB2B6869614
:10B7D000A6D0CAF349DAA6CBF8D8B0B4B8D8AD84AD
:10B7E000F2C0DFF18FCBC3A8B2B68696C8C1CBC377
:10B7F000F3B0B48898A821DB718D9D71859521D90E
:10B80000ADF2FAD88597A828D9F408D8F28D29DAAC
:10B81000F405D9F285A4C2F2D8A88D9401D1D9F447
:10B8200011F2D88721D8F40AD8F28498A8C801D197
:10B83000D9F411D8F3A4C8BBAFD0F2DEF8F8F8F809
:10B84000F8F8F8F8D8F1B8F6B5B9B08A95A3DE3CA7
:10B85000A3D9F8D85CA3D9F8D87CA3D9F8D8F8F93B
:10B86000D1A5D9DFDAFAD8B18530F7D9DED8F830EA
:10B87000ADDADED8F2B48C99A32D557DA083DFDF3D
:10B88000DFB591A0F629D9FBD8A0FC29D9FAD8A018
:10B89000D051D9F8D8FC51D9F9D879D9FBD8A0D052
:10B8A000FC79D9FAD8A1F9F9F9F9F9A0DADFDFDFE3
:10B8B000D8A1F8F8F8F8F8ACDEF8ADDE8393AC2C3C
:10B8C000547CF1A8DFDFDFF69D2CDAA0DFD9FADBAC
:10B8D0002DF8D8A850DAA0D0DED9D0F8F8F8DB558A
:10B8E000F8D8A878DAA0D0DFD9D0FAF8F8F8F8DBE1
:10B8F0007DF8D89CA88CF530DB38D9D0DEDFA0D01D
:10B90000DEDFD8A848DB58D9DFD0DEA0DFD0DED814
:10B91000A868DB70D9DFDFA0DFDFD8F1A888902C22
:10B92000547C98A8D05C38D1DAF2AE8CDFF9D8B06C
:10B9300087A8C1C1B188A8C6F9F9DA36D8A8F9DA5A
:10B9400036D8A8F9DA36D8A8F9DA36D8A8F9DA3626
:10B95000D8F78D9DADF818DAF2AEDFD8F7ADFA3032
:10B96000D9A4DEF9D8F2AEDEFAF983A7D9C3C5C7E8
:10B97000F1889BA77AADF7DEDFA4F8849408A79737
:10B98000F300AEF29819A488C6A39488F632DFF2C9
:10B990008393DB09D9F2AADFD8D8AEF8F9D1DAF36C
:10B9A000A4DEA7F1889B7AD8F38494AE19F9DAAAB9
:10B9B000F1DFD8A881C0C3C5C7A39283F628ADDE46
:10B9C000D9F8D8A350ADD9F8D8A378ADD9F8D8F81C
:10B9D000F9D1A1DADEC3C5C7D8A18194F818F2B0B5
:10B9E00089ACC3C5C7F1D8B8B4B09786A8319B0657
:10B9F0009907AB9728889BF00C201440B0B4B8F09E
:10BA0000A88A9A285078B79BA8295179247059445C
:10BA10006938644831F1BBAB88002C547CF0B38B9F
:10BA2000B8A804285078F1B088B49726A85998BBD4
:10BA3000ABB38B02264666B0B8F08A9CA829517930
:10BA40008B2951798A2470598B2058718A4469381E
:10BA50008B3940688A6448318B30496088F1AC008A
:10BA60002C547CF08CA804285078F1889726A8598B
:10BA700098AC8C02264666F0899CA82951792470DE
:10BA800059446938644831A98809205970AB113884
:10BA90004069A8193148608CA83C415C207C00F1C9
:10BAA00087981986A86E767EA999882D557DD8B17C
:10BAB000B5B9A3DFDFDFAED0DFAAD0DEF2ABF8F995
:10BAC000D9B087C4AAF1DFDFBBAFDFDFB9D8B1F1EE
:10BAD000A3978E60DFB084F2C8F8F9D9DED89385D9
:10BAE000F14AB183A308B5839A0810B79F10D8F123
:10BAF000B0BAAEB08AC2B2B68E9EF1FBD9F41DD8F0
:10BB0000F9D90CF1D8F8F8AD61D9AEFBD8F40CF145
:10BB1000D8F8F8AD19D9AEFBDFD8F416F1D8F8ADE6
:10BB20008D61D9F4F4ACF59C9C8DDF2BBAB6AEFADE
:10BB3000F8F40BD8F1AED0F8AD51DAAEFAF8F1D88E
:10BB4000B9B1B6A3839C08B9B1839AB5AAC0FD3038
:10BB500083B79F10B58B93F20202D1ABDADED8F136
:10BB6000B080BAABC0C3B284C1C3D8B1B9F38BA3A0
:10BB700091B609B4D9ABDEB0879CB9A3DDF1B38B24
:10BB80008B8B8B8BB087A3A3A3A3B28BB69BF2A3A3
:10BB9000A3A3A3A3A3A3A3A3A3F1B087B59AA3F3DD
:10BBA0009BA3A3DCBAACDFB9A3A3A3A3A3A3A3A3C2
:10BBB000A3A3A3A3A3A3A3A3D8D8D8BBB3B7F1AA25
:10BBC000F9DAFFD9809AAA28B48098A720B7978776
:10BBD000A86688F07951F1902C870CA78197629321
:10BBE000F071716085940129517990A5F1284C6C10
:10BBF000870C95188578A38390284C6C886CD8F3B3
:10BC0000A28200F210A8921980A2F2D926D8F18857
:10BC1000A84DD948D896A83980D93CD89580A8395C
:10BC2000A68698D92CDA87A72CD8A8899519A98037
:10BC3000D938D8A88939A980DA3CD8A82EA8399053
:10BC4000D90CD8A8953198D90CD8A809D9FFD80112
:10BC5000DAFFD89539A9DA26FFD890A80D8999A8D6
:10BC600010809821DA2ED88999A83180DA2ED8A8A8
:10BC700086963180DA2ED8A8873180DA2ED8A8822D
:10BC800092F34180F1D92ED8A882F31980F1D92EF0
:10BC9000D882ACF3C0A28022F1A62EA72EA92298AA
:10BCA000A829DAACDEFFD8A2F22AF1A92E8292A846
:10BCB000F23180A696F1D900AC8C9C0C30ACDED071
:10BCC000DEFFD88C9CACD010ACDE8092A2F24C820D
:10BCD000A8F1CAF235F19688A6D900D8F1FF010083
:10BCE00002000400060008000A000C0010002000FA
:10BCF0004000800000010101010307010000080469
:10BD00000204080101010000000001020304010215
:10BD10000304060708090000555555555555C53FFC
:10BD20007D6FEB0312D6D4BF5544880E55C1C93F71
:10BD30003B8F68B52882A4BF88B20175E0EF493F08
:10BD400009F7FD0DE13D023F4B2D8A1C273A03C048
:10BD5000C88A599CE52A004059018D1B6C06E6BF34
:10BD600082922EB1C5B8B33F4FBB610567ACDD3FD2
:10BD7000182D4454FB21E93F9BF681D20B73EF3F12
:10BD8000182D4454FB21F93FE2652F227F2B7A3C8A
:10BD9000075C143326A6813CBDCBF07A8807703C43
:10BDA000075C143326A6913CC4EB98999999C9BFB6
:10BDB000711623FEC671BCBF6D9A74AFF2B0B3BFEB
:10BDC0009AFDDE522DDEADBF2F6C6A2C44B4A2BFAB
:10BDD0000D5555555555D53FFF8300922449C23F17
:10BDE0006E204CC5CD45B73F513DD0A0660DB13F4B
:10BDF000EB0D76244B7BA93F11DA22E33AAD903F5D
:10BE0000000000000000000050726F647563742031
:10BE100049442072656164206173203020696E643A
:10BE2000696361746573206465766963652069730D
:10BE30002065697468657220696E636F6D706174E6
:10BE400069626C65206F7220616E204D50553330F1
:10BE500035302E0A0000000078BE000800000024E3
:10BE600064000000D87D0008DCBE000864000024E7
:10BE700044070000E87D000894B00008B2B0000854
:10BE800000000000000000000000000000000000B2
:10BE900000000000000000000000000000000000A2
:10BEA000C0B0000800FF000000FF0000000100001B
:10BEB00068000000D1000000D00000000100000078
:10BEC0000000000010000000010000000090D003FE
:0CBED0000090D003000000000000000003
:040000050800029954
:00000001FF
